:090000000217FC0247FC25730005
:10000B00024932E4FFFE120731600C0FEF70010E54
:0F001B0009E970F20A80EF220249415322E022E4
:07002B00024FFC43EA4022F2
:100033000274269000E27406F09000E07400F090E1
:1000430000E27412F07581AA1238370217FC75A802
:10005300009000E27406F09000E07480F09000E2FB
:10006300740CF00217FC244750524D430000020465
:1000730037E86480F8E933E83360110460F0ED3366
:10008300EC337009E8FCE9FDEAFEEBFF220460DED5
:10009300D3EB9FEA9EE99DE8C2E78CF0C2F795F0A7
:1000A300400CE8CCF8E9CDF9EACEFAEBCFFB120429
:1000B3000285D0F05804700320D5B3E804700750CC
:1000C30002B2D502044192D5EC0460F7E4CCC0E05F
:1000D300C398F8603B94186008400DD0E0FB02041D
:1000E30019E4FBFAC9FC8028E830E406E4C9FBE420
:1000F300CAFCE830E305E4C9CACBFCE85407601046
:10010300F8C3E913F9EA13FAEB13FBEC13FCD8F188
:1001130030F52FC3E49CFCEF9BFFEE9AFEED99FDB7
:10012300D0E0FBEF4E4D4C701222DB0302043EEC99
:100133002CFCEF33FFEE33FEED33FDED30E7EB0246
:100143000419EF2BFFEE3AFEED39FDD0E0FB50131F
:100153000BBB0003020441ED13FDEE13FEEF13FF8F
:10016300EC13FC020419EC4D6011E8497017ED33F0
:10017300EC3304600DE4FCFFFEFD22E933E83304B5
:1001830070F802043712040258046009E4CC248195
:10019300500628500902044128400302043EC0E0EF
:1001A300EB4A7044B98006D0E0FB02042DEF4E7099
:1001B3001CBD8008EBFFEAFEE9FD80EBE98DF0A4AE
:1001C300FEE5F0020252E9CDF9EAFEEBFFEF89F01A
:1001D300A4FCE5F0CE89F0A42EFFE435F0CD89F040
:1001E300A42DFEE435F08067EF4E7005BD80D78007
:1001F300C3EF8BF0A4ACF0EE8BF0A42CFCE435F051
:10020300F8EF8AF0A42CE5F038FCE433CB8DF0A4AE
:100213002CFCE5F03BF8EE8AF0A42CFCE5F038F872
:10022300E433CF89F0A42CFCE5F038CF3400CE8939
:10023300F0A42FFFE5F03EFEE433C98DF0A42EFEBB
:10024300E5F039CD8AF0A42FFFE5F03EFEE43DFD55
:1002530033D0E0FB50070BBB000F020441EC2CFC36
:10026300EF33FFEE33FEED33FD020419020441ECDC
:100273005D046005E8590470030204371204025850
:100283000460F6EC4860F2EC7004FDFEFF22C860E7
:10029300DB2481C85009C3986002500602043E98CB
:1002A30050CAF582E9294B4A7005AB8202042D75C9
:1002B300F0007C1A7880C3EF9BEE9AED99400DC352
:1002C300EF9BFFEE9AFEED99FDE842F0DC23ACF0E4
:1002D300D0E0FFD0E0FED0E0FDAB8220E7101BEBC7
:1002E30060BAEC2CFCEF33FFEE33FEED33FD02047A
:1002F30019E803F830E705C0F075F000EF2FFFEEC3
:1003030033FEED33FD40B830E7C280AA74F8CC6405
:1003130080CCC86480C8F582046043C3EB9FF5F0CA
:10032300EA9E42F0E99D42F0E89C45F060305018A7
:10033300E5825FFFE582F42B5582FB50210ABA0068
:100343001D09B90019088016E5825BFBE582F42FCD
:100353005582FF50090EBE00050DBD00010CC3EB15
:100363009FF5F0EA9E42F0E99D42F0E89C45F0607B
:1003730007CC4820E701B3EC22ED33EC33600A04E9
:100383007003BD8004ECB2E7FC2275F020800E758B
:10039300F010800575F0087D007E007F003392D554
:1003A30030D503120959EC334010EF33FFEE33FE1F
:1003B300ED33FDEC33FCD5F0ED22E5F0247EA2D540
:1003C30013CC92E7CDCEFF22EDD2E7CD33EC3392BF
:1003D300D524814006E4FFFEFDFC22FCE4CFCECD14
:1003E300CC24E0501174FF80EDC3CC13CCCD13CDDE
:1003F300CE13CECF13CF0470F030D5DE020959E906
:10040300D2E7C933E833F892D5EDD2E7CD33EC33F5
:10041300FC5002B2D522EC30E7100FBF000C0EBE29
:1004230000080DBD00040BEB6014A2D5EB13FCED2B
:1004330092E7FD2274FFFCFDFEFF22E480F8A2D5C3
:1004430074FF13FC7D80E480EFC0E0EFFBEEFAED78
:10045300F9ECF8120169D0E0F5F0EFFBEEFAEDF9F3
:10046300ECF8120997A3A3A3A3E8C0E0E9C0E0EA6C
:10047300C0E0EBC0E0C0F01201691209B4A3A3A36A
:10048300A3120078D0F0D0E0FBD0E0FAD0E0F9D0AE
:10049300E0F8D5F0D4223F8000004120000042C89C
:1004A3000000447A0000461C400047C350004974D2
:1004B30024004B1896804CBEBC205A0E1BCA6753AF
:1004C300C21C749DC5AEFB60065407601C23231237
:1004D30004F7EB543860091204E31204F2120169C1
:1004E300ECF8EDF9EEFAEFCB22EB1204F280F154C3
:1004F3003803241C900499FE93FC0EEE93FD0EEE3C
:10050300930ECE93FF22F920E72824F950037907AD
:10051300E4F42402FB18DBFDE624FB5014E9600D30
:10052300E4F618E604F6B40A08E4F6D9F57401F61D
:100533000A22C2D522ED33EC3392D5FA602AB4FFF6
:1005430033EDC2E77BFF60067A05795DE4227A0525
:10055300796620D5047A057961224E614E002B49D4
:100563004E46002D494E4600E47A08F608DAFC7B35
:1005730000740722E8C0E0ECC0E0EDC0E0EEC0E0AC
:10058300EFC0E0EA75F010A4CAABF075F04DA42BF0
:10059300FBE435F0FCEA2410FAEB34C5FBEC34D968
:1005A300FCEDC2E7FF75F056A4F42411C5F0F43452
:1005B300C58FF0A42AE5F03BE43CF620E7141204CF
:1005C300C9D0E0FFD0E0FED0E0FDD0E0FC12027223
:1005D3008014F4041204C9D0E0FFD0E0FED0E0FDA3
:1005E300D0E0FC120169D0E0F8E6FAEDD2E7CD33B2
:1005F300EC332482FBE4C3CF33CFCE33CECD33CD24
:1006030033DBF37B0775F00A846004F6081B0AE505
:10061300F0F6088FF0740AA4FFACF08EF0740AA40D
:100623002CFEACF050010C8DF0740AA42CFDE435C3
:10063300F0F608DBDE740722E709F608DFFA8046E6
:10064300E709F208DFFA803E88828C83E709F0A38A
:10065300DFFA8032E309F608DFFA8078E309F2086B
:10066300DFFA807088828C83E309F0A3DFFA806469
:1006730089828A83E0A3F608DFFA805889828A8315
:10068300E0A3F208DFFA804C80D280FA80C680D4DF
:10069300806980F28033801080A680EA809A80A8E7
:1006A30080DA80E280CA803389828A83ECFAE49319
:1006B300A3C8C582C8CCC583CCF0A3C8C582C8CCA7
:1006C300C583CCDFE9DEE7800D89828A83E493A3C7
:1006D300F608DFF9ECFAA9F0EDFB2289828A83ECB4
:1006E300FAE0A3C8C582C8CCC583CCF0A3C8C58231
:1006F300C8CCC583CCDFEADEE880DB89828A83E469
:1007030093A3F208DFF980CC88F0EF60010E4E600E
:10071300C388F0ED2402B4040050B9F582EB24023F
:10072300B4040050AF232345822390068B73BB018F
:100733000689828A83E0225002E722BBFE02E3227B
:1007430089828A83E49322BB010CE58229F582E541
:10075300833AF583E0225006E92582F8E622BBFEC0
:1007630006E92582F8E222E58229F582E5833AF556
:1007730083E49322BB010689828A83F0225002F725
:1007830022BBFE01F322EF8DF0A4A8F0CF8CF0A4DE
:1007930028CE8DF0A42EFE22BC000BBE0029EF8DC7
:1007A300F084FFADF022E4CCF875F008EF2FFFEEF4
:1007B30033FEEC33FCEE9DEC984005FCEE9DFE0F02
:1007C300D5F0E9E4CEFD22EDF8F5F0EE8420D21C5D
:1007D300FEADF075F008EF2FFFED33FD40079850A5
:1007E30006D5F0F222C398FD0FD5F0EA22C2D5EC6C
:1007F30030E709B2D5E4C39DFDE49CFCEE30E71578
:10080300B2D5E4C39FFFE49EFE12079BC3E49DFDA4
:10081300E49CFC800312079B30D507C3E49FFFE4ED
:100823009EFE22A3F8E0C5F025F0F0E58215827064
:10083300021583E0C838F0E822E88FF0A4CC8BF0EF
:10084300A42CFCE98EF0A42CFC8AF0EDA42CFCEA89
:100853008EF0A4CDA8F08BF0A42DCC3825F0FDE9C3
:100863008FF0A42CCD35F0FCEB8EF0A4FEA9F0EBB9
:100873008FF0A4CFC5F02ECD39FEE43CFCEAA42DC5
:10088300CE35F0FDE43CFC2275F008758200EF2FB5
:10089300FFEE33FECD33CDCC33CCC58233C5829B43
:1008A300ED9AEC99E58298400CF582EE9BFEED9A69
:1008B300FDEC99FC0FD5F0D6E4CEFBE4CDFAE4CC05
:1008C300F9A88222B800C1B90059BA002DEC8BF007
:1008D30084CFCECDFCE5F0CBF97818EF2FFFEE33C4
:1008E300FEED33FDEC33FCEB33FB10D703994004EF
:1008F300EB99FB0FD8E5E4F9FA227818EF2FFFEE16
:1009030033FEED33FDEC33FCC933C910D7059BE946
:100913009A4007EC9BFCE99AF90FD8E0E4C9FAE4A2
:10092300CCFB2275F010EF2FFFEE33FEED33FDCC41
:1009330033CCC833C810D7079BEC9AE899400AED2B
:100943009BFDEC9AFCE899F80FD5F0DAE4CDFBE4D3
:10095300CCFAE4C8F922C3E49FFFE49EFEE49DFDC4
:10096300E49CFC22EB9FF5F0EA9E42F0E99D42F005
:10097300E89C45F022E8600FECC313FCED13FDEE99
:1009830013FEEF13FFD8F122E6FC08E6FD08E6FEAE
:1009930008E6FF22E493FC740193FD740293FE7452
:1009A3000393FF22E6FB08E6F908E6FA08E6CBF82C
:1009B30022E493F8740193F9740293FA740393FB9A
:1009C30022ECF608EDF608EEF608EFF622ECF0A3BB
:1009D300EDF0A3EEF0A3EFF022A42582F582E5F07B
:1009E3003583F58322FAE6FB0808E6F925F0F618C5
:1009F300E6CA3AF622D083D082F8E49370127401E7
:100A030093700DA3A393F8740193F5828883E47321
:100A13007402936860EFA3A3A380DF8A838982E4CF
:100A230073EF4E6012EF60010EEDBB010B89828AFA
:100A330083F0A3DFFCDEFA2289F05007F709DFFC1D
:100A4300A9F022BBFEFCF309DFFCA9F022E5602438
:100A53004CF8E60560227849302F02784CE475F0B3
:100A6300011209E80207312028EB7F2ED2288018D3
:100A7300EF540F2490D43440D4FF302C0BEF24BF19
:100A8300B41A0050032461FFE56160021561056437
:100A9300E56470020563302F0D7849E475F00112A7
:100AA30009E8EF020777021A0C7403D22F8003E4DC
:100AB300C22FF5608B498A4A894BE4F561F563F5EA
:100AC30064E56160077F20120A8B80F57562FFC2BF
:100AD30029C228C22AC22BC22DC22EC230120A59E1
:100AE300FF700D302F057F00120A9CAF64AE6322A6
:100AF300B4255FC2D5C22C120A59FF24D0B40A0010
:100B0300501A75F00A786130D50508B6FF0106C69C
:100B1300A426F620D5047002D22B80D924CFB41A90
:100B230000EF5004C2E5D22C020D89D22980C6D22F
:100B33002880C0D22A80BCD2D580BAD22D80B47F7F
:100B430020120A8B202A077401B5610040F1120AB2
:100B530050FF120A8B020AC4D230D22E8095120A99
:100B630050FB120A50FA120A50F94A4B7006798068
:100B73007A0E7BFF202A2EE561602A7E008E827525
:100B8300830012074A60060EEE656270F0C2D5EB71
:100B9300C0E0EAC0E0E9C0E0EE120DE9D0E0F9D030
:100BA300E0FAD0E0FB120731FF60AAEBC0E0EAC035
:100BB300E0E9C0E0120A8BD0E02401F9D0E0340070
:100BC300FAD0E0FBE5620460DCD562D98087D22AE3
:100BD30080A2120DCC60F7E562700104120509A929
:100BE30062600DE562600914F562120E73EF60F343
:100BF300EA30E702F404C3995077EAF4256204303B
:100C0300E701E404F562800D120DCC60C1EA0562D0
:100C13002562120509EA785FF630E701E4256204EC
:100C2300D56204202D0114120DE9E4C0E0120E7305
:100C3300785FE6601320E70714F6120A7380220434
:100C4300F6D0E014C0E07F00120A73E56260071279
:100C53000A6A1562800B302D03120A6AD0E0020A79
:100C6300C4D0E00480C5120DCC60A0E56204120577
:100C730009785FEAF6E562202D026001042404127C
:100C83000DE974FF04C0E0120E73120A73E56220CB
:100C93002D026003120A6AD0E0B562E87F45120AAA
:100CA3007D785FE67F2B30E7047F2DF404C0E012EC
:100CB3000A8BD0E075F00A84C0F0120A74D0E012F7
:100CC3000A74020AC4791080027908C22EC23080E5
:100CD30008D2D5790A8004790AC2D5E56204700284
:100CE300F562E4FAFDFEFF120A50FC7B082029138B
:100CF300120A50FD7B1030280A120A50FE120A50C5
:100D0300FF7B20EC3382D592D55013C3E430280601
:100D13009FFFE49EFEE42029039DFDE49CFCE4CBBD
:100D2300F8C229EC700CCFCECDCCE824F8F870F3E0
:100D33008017C3EF33FFEE33FEED33FDEC33FCEBF3
:100D430033FB994002FB0FD8E9EB302905F8D0E0DB
:100D5300C448B229C0E00AEC4D4E4F78207B0070A6
:100D6300C2EAB5620040BCC0E0120DEBD0F0D0E0A7
:100D7300202904C4C0E0C4B229C0F0120A74D0F020
:100D8300D5F0EB020AC41209F80B61530CC8580BD7
:100D9300324C0B2E420CCC4F0CD4440CD4490B4791
:100DA300430CDA550C0B460C69450BD5470EA05086
:100DB3000B362D0B3A2E0B5D2B0B3E230B5B200EBC
:100DC300892A0AF64800000B55E562B4FF037562F1
:100DD30006120A50FC120A50FD120A50FE120A5063
:100DE300FF7858020538790AA2D5202B14302D0933
:100DF300B910020404B9080104A2D5202E0250013F
:100E030004202A68922AB561005034C0E07F203064
:100E13002B197F30A22A722E722D500F120E42C24E
:100E23002AC22EC22DC2307F30800F302D03E9C07D
:100E3300E0120A8B302D03D0E0F9D0E0B561CC305D
:100E43002D177F30B9100C120A8B7F58302C077F77
:100E5300788003B90803120A8B302A057F2D020A12
:100E63008B7F202030F87F2B202EF322922A80CFF5
:100E73007F00B4070050052458F8E6FF22286E755A
:100E83006C6C2900D229120A503029F8C2297861E2
:100E930030D50108F6020AF62D50434958120A507C
:100EA3002403B405004001E4900E9B93120A7C7462
:100EB3003A120A7CD22B756104020CC825730020F8
:100EC3002573003E005F2573002020202020202072
:100ED3002020202020202020004B4D480025337562
:100EE300004D5048003C005F257320202020202027
:100EF300202020202020002530337520004C415431
:100F03005F3A5F25635F25303375405F2530322EAE
:100F13003032662720004C4F4E5F3A5F25635F25D2
:100F2300303375405F2530322E303266272000443F
:100F330049525F3A5F2530337540002533627500AF
:100F43005E0025733A2025362E3166204D69002533
:100F5300733A2025362E3166204B4D0025733A20F7
:100F6300252D322E316600560025733A20256278EE
:100F73002E253162780025733A20002562752F25CE
:100F830062752F25347500204B204D204820284BB7
:100F93004D2F482900204D2050204820284D494CF2
:100FA300452F482900474D5420202B2562642000FB
:100FB300474D54202025626420200044455341437B
:100FC30054495641444F5300414354495641444FB9
:100FD300532020200053454C2E50414E54414C4C3D
:100FE300412020202020004C494D2E56454C4F4394
:100FF30049444144202020200050554E544F535F14
:101003005553554152494F20202000494C554D49D5
:101013004E414349674E20202020202000434F4E5D
:101023004649475F50414953202020202020004952
:101033004E464F5F44454C5F53495354454D412001
:101043000020554E49444144455320202020202070
:101053002000204855534F20484F524152494F20BA
:1010630020200020415649534F5320534F4E4F5297
:101073004F532000FF6F1FFF561AFF4DB4FF70132D
:10108300FF5136FF3C96FF56D1FF70E6FF578301B1
:10109300220001200001230001210041881800449F
:1010A300880E000000004188190041880C00418827
:1010B30017004188150041880D0041880A004186C8
:1010C300210041851F00418520004487370000002F
:1010D300004A874D000000000000000000004A871E
:1010E300430000000000000000000044872D0000C2
:1010F300000042872B000044873300000000418733
:10110300310041875D004287200000418732004261
:10111300875B1C204487220000000041872900418F
:10112300872A004187280044875E0000000041872A
:1011330063004187640041876200448757000000D1
:101143000044871C0000000044873F00000000416A
:10115300872600418727004A8765000000000000BA
:101163000000FF004A87730000000000000000FF3A
:101173000042877D000042878D00004E877F00007C
:101183000000000000000000000000004187900004
:1011930041878F0044876F0000000044879100005F
:1011A30000004A882B0000000000000000FF0042FE
:1011B300883500004A88370000000000000000FF67
:1011C3000042884100004987CF000502010504025F
:1011D30005064987C6000502010504020506418785
:1011E300D9004187D8004287DA00004187DC0056E6
:1011F30087DF000000005600000000000000000030
:10120300000000FF0000000002A4862202A686223E
:101213004C87FD1F1C1F1E1F1E1F1F1E1F1E1F414D
:10122300841B0002A8000041884300418844FF0159
:10123300AA004188450041884700418846000124AF
:10124300000025730025336275005E004E4525338B
:10125300750045202533750053452533750053200C
:101263002533752A00534F253375004F20253375D9
:10127300004E4F253375004E202533750025336C02
:1012830075004D00202020203E002020203E3E00FF
:1012930020203E3E3E00203E3E3E3E003E3E3E3E41
:1012A3003E0025732020200025733E202000257357
:1012B3003E3E200025733E3E3E00253475004D50D2
:1012C30048004B4D48004E452533754000452025C9
:1012D300337540005345253375400053202533753E
:1012E3004000534F25337540004F20253375400090
:1012F3004E4F25337540004E202533754000202086
:10130300202020400025352E3166204D69002535EB
:101313002E3166204B4D00253262753A25303262FC
:1013230075002573253262753A2530326275007E69
:101333000025362E3166204D690025362E31662074
:101343004B4D00253375204D504800253375204BF8
:101353004D480025342E3166204D50480025342E4B
:101363003166204B4D4800253262752F2532627558
:101373000025733A252D322E316656004241540022
:1013830025352E31664D690025352E31664B4D00CE
:101393002533754D5048002533754B4D4800253393
:1013A300750045584345534F002532750051756903
:1013B3006E74657A7A00414C455254455200257348
:1013C30020475053002573204F4B202120202020FD
:1013D3002020003A70FA83BCAAE9E43E81E0F8BF1A
:1013E3009DE9E63F80000039283C1ABB9969663DB8
:1013F300A335E3BF255DE73FC90FDB418DDBCCC4DC
:101403004936EE45C9913FC5B0F83D3F800000C362
:1014130017F534452FFA73C60AFDDD1214C504A26D
:10142300E192281420E0159013D6740412044C8022
:10143300261214C530E102B22820E0EB8C278D2858
:101443008E298F2A9013EA740412044CA827A92822
:10145300AA29AB2A120169ED4C6007302804EC6419
:1014630080FC221214C5C0E08C278D288E298F2A78
:1014730090140E740312044CA827A928AA29AB2A96
:10148300120169ECC527FCEDC528FDEEC529FEEF69
:10149300C52AFF9013FE740312044CD082A827A917
:1014A30028AA29AB2AE58230E007120272B228800B
:1014B300A6EFCBFFEECAFEEDC9FDECC8FC1202722B
:1014C3008095ED33EC547FCC33922824605007D0C1
:1014D300E0D0E00204377B837AF97922783E120167
:1014E30069EDF933ECF83324815011EFFBEEFA1276
:1014F30003CB12038DECB2E7FC120078ED33EC332F
:10150300602F2403F8C313FCED92E7FDE82481E484
:10151300501FECF8EDF9EEFAEFFB1203CBEF04C228
:10152300E0FCF582120397ECB2E7FC120078E58247
:1015330003FAED33EC3360071413FCED92E7FDEA95
:1015430022BE1249253E4CCCCDBEAAAAAB3F800099
:10155300003E7ADBB03EED63383F24BC7D3F490F4C
:10156300DBED33ECC2E7CC339228B4FF13ED547FA9
:1015730060030204377FDB7E0F7DC97C3F02165F69
:10158300C229C3947F401E7007EDD2E794904015A3
:10159300EFFBEEFAEDF9ECF87F007E007D807C3FF7
:1015A300120272D229ED33EC33248430E705E4C010
:1015B300E0806D04FAEDD2E754F0C333DAFD54074B
:1015C30034002323C0E0CCC0E0F8EDC0E0F9EEC066
:1015D300E0FAEFC0E0FBE4120397EC24FEFC8C3846
:1015E3008D398E3A8F3B1201697B007A00798078BE
:1015F3003F120078ECC538B2E7FCEDC539FDEEC506
:101603003AFEEFC53BFFD0E0FBD0E0FAD0E0F9D0E3
:10161300E0F8120078A838A939AA3AAB3B12027253
:101623008C388D398E3A8F3B901544740312044CD9
:10163300A838A939AA3AAB3B120169D0E0600F245C
:1016430050F582E43415F5831209B4120078302979
:101653000B7BDB7A0F79C978BF120078ED33EC335B
:101663006006ECA22892E7FC22C229C22AC22BC23E
:101673002CF9E4F52EF52FFCFDFEFFE91028EA20F6
:101683002B0CB42D04D22BD322B42B02D32224D07F
:10169300504794095041240A302C15F8852FF074D3
:1016A3000AA42872E74051C5F0704D85F02FD3226C
:1016B300D22AC0E0E4FBFA79207841120169ECF800
:1016C300EDF9EEFAEFFBD0E0FCE412039712007899
:1016D3003029B4152ED322240A202C20B4FE07204F
:1016E300291AD229D32224EB600424E0700EA22B02
:1016F3009229D22CC22BD322C3020437E4302C0B01
:10170300E52F302B02F404A229922B302AEA252E4E
:1017130020D2E5A2E7922C5002F404B4260050D85C
:10172300CCC0E0EDC0E0EEC0E0EFC0E0EC1204C9D5
:10173300D0E0FFD0E0FED0E0FDD0E0FC202C05128D
:1017430001698003120272302B0312037CC322024D
:10175300043722EDA2E7D2E7F9EC3340F260F3B4A9
:10176300FF08ED547F70E8020441F82481C2E0C011
:10177300E0F40428FAC313FCED92E7FD8C308D31BD
:101783008E328F33EEA2E7E9BA7F02C3133400949B
:1017930000FA75F091A4E5F013F494FE8AF0A433F3
:1017A300E5F033248CD313FDE492E7FE7F007C3F06
:1017B300758302ECC0E0F8EDC0E0F9EEC0E0FAEFAB
:1017C300C0E0FBAC30AD31AE32AF33120272D0E0C9
:1017D300FBD0E0FAD0E0F9D0E0F8120078ED6480B5
:1017E300FD30E7011CD583CBED33CC33F8D0E0A239
:1017F300E71328C313CC13FD227581AA02183D02F7
:101803003154E493A3F8E493A34003F68001F20870
:10181300DFF48029E493A3F85407240CC8C333C42A
:10182300540F4420C8834004F456800146F6DFE495
:10183300800B0102040810204080901092E47E0186
:101843009360BCA3FF543F30E509541FFEE493A308
:1018530060010ECF54C025E060A840B8E493A3FA1A
:10186300E493A3F8E493A3C8C582C8CAC583CAF0A6
:10187300A3C8C582C8CAC583CADFE9DEE780BE8FB5
:10188300338E328D318C30AB37AA36A935A834125A
:1018930002721215648F338E328D318C30E5343001
:1018A300E747ECC0E0EDC0E0EEC0E0EFC0E0E4FFEE
:1018B300FEFDFCAB33AA32A931A83012030F7BDB48
:1018C300600250087A0F7949784080067A0F794987
:1018D30078C0D0E0FFD0E0FED0E0FDD0E0FC120005
:1018E300788F338E328D318C30AF33AE32AD31AC35
:1018F30030228B278A288929AB2AAA2BA92C1207E5
:1019030031FEAB27AA28A929120731FF6E702BEFEE
:10191300600DE52E152E7002152D14452D70037FD5
:10192300002274012529F529E43528F528740125B9
:101933002CF52CE4352BF52B80BEAB27AA28A9293F
:10194300120731FFD3EE6480F8EF64809840037F81
:1019530001227FFF22D2288B2B8A2C892D121994E6
:10196300C0E0FF121A4ED0E040F312167F4001226E
:10197300ECC0E0EDC0E0EEC0E0EFC0E0121994D09F
:10198300F0AFF0D0F0AEF0D0F0ADF0D0F0ACF0802E
:10199300D9E475F001782B1209E8020731257300A9
:1019A3005350454544005253002533754D5048006C
:1019B3002533754B4D48004C41534552003E3E3E46
:1019C300004B412042414E4400256264004B2042BB
:1019D300414E4400582042414E440085434C8544C7
:1019E3004D85454EEBC546FBEAC547FAE9C548F9BF
:1019F3007F09784F120731F60809E970010ADFF40D
:101A0300AB46AA47A948020AACEFB40A07740D1201
:101A13001A17740A309811A899B8130CC298309801
:101A2300FDA899C298B811F63099FDC299F599228B
:101A3300253375002573004E49694F532121210039
:101A4300502E4E4547524F21212100EFC3940940A8
:101A530005EF940E4003BF2003D38001C3222573F7
:101A63000025733A2575005F564F4C554D454E2062
:101A73002020202020202000434F4E454354415234
:101A83005F4750530056454C2E00414C41524D4147
:101A930000414354495641442E0044455341435465
:101AA300495641444F530043644D4152410042491A
:101AB3004449524543432E0043414D494E4F202054
:101AC300202000434F4E54524F4C0046494E202095
:101AD300202000534954494F0050454C4947524F29
:101AE300534F004144564552542E0050554E544FC7
:101AF300005F5553554152494F00416941444944A0
:101B03004F004C4C454E4F0053555052494D49449C
:101B13004F00564143664F004D454E685F50524952
:101B23004E434950414C005F53454C45434349673D
:101B33004E5F4D4F444F2020004C494D49544500C2
:101B43004C494D495445005F494C4C554D494E4114
:101B53004349674E20202000414A555354455F5066
:101B6300416653202020202000494E464F5F4445C4
:101B73004C5F53665354454D41005F554E494441B4
:101B8300442020202020202020200055534552208F
:101B9300494E464F004855534F20484F52415249F2
:101BA3004F202000415649534F5300415649534F4C
:101BB3005320534F4E4F524F5320005245414A55E5
:101BC300535445005452415945432E00444546451C
:101BD30043544F00444554414C4C455300434F4EEE
:101BE300464F525400532820004E4F200042525576
:101BF3004A554C41004F444F004645434841005429
:101C030065636E6F6C6F67236100202054455354E6
:101C130020200053494E2050554E544F53005452E8
:101C230041594543544F200050494C412020202026
:101C330000534F465457415245004441544F53209B
:101C4300202000475541524441444F202000505525
:101C53004E544F2044452055534152494F00522F73
:101C63004F444F004D45444941005449454D2E00D2
:101C730000000000000000004F4F000000060006B7
:101C8300000000487A410000F8252524F800007F71
:101C930025251A007D4140417D000000000B07000F
:101CA30000487A490000F824252525F8030300009D
:101CB300000008083E080800000000583800080823
:101CC300080808000000400000002010080402007B
:101CD3003E5149453E0000427F4000004261514968
:101CE30046002241494936001814127F1000274547
:101CF300454539003C4A4949300001710905030053
:101D0300364949493600064949291E00003636003E
:101D13000000005B3B00000000081C3E7F00141421
:101D2300141414007F3E1C08000002015909060028
:101D3300324959413E007E1111117E00417F4949CC
:101D430036003E4141412200417F41413E007F49EF
:101D5300494141007F09090901003E4149497A008F
:101D63007F0808087F0000417F4100002040413F79
:101D730001007F08142241007F40404040007F0261
:101D83000C027F007F0204087F003E4141413E0078
:101D93007F09090906003E4151215E007F09192987
:101DA300460026494949320001017F0101003F40B5
:101DB30040403F000718601807003F4038403F008D
:101DC300631408146300070870080700615149454C
:101DD3004300007F4141000002040810200000413D
:101DE300417F0000040201020400404040404000E3
:101DF3000004020100002054545478007F484444F6
:101E03003800384444442000384444487F00385460
:101E130054540800087E09020000081454543C007E
:101E23007F080404780000447D4000002040443DC6
:101E33000000007F1028440000417F400000780428
:101E4300180478007C0804047800384444443800BB
:101E53007C14242418001824147C4000007C0804FB
:101E63000400485454542000043E442000003C40E5
:101E730040207C001C2040201C003C4030403C00A3
:101E83004428102844004C5050503C004464544CA7
:101E930044000008364100000000770000000041C4
:101EA300360800000804081008002A552A552A009D
:101EB3000800000000000000000000000000000017
:101EC300000400F8F800000D0D000638380038381B
:101ED300000000000000000820F8F820F8F82000B7
:101EE300020F0F020F0F0200003078CE8E18100081
:101EF30000040C38390F060008183C24BCD86030A5
:101F0300000006030E1E121E0C0800B0F8487830BD
:101F1300000000070F0809070F0902383800000402
:101F2300E0F81C04030F1C1004041CF8E0101C0F41
:101F3300030780A0E0C0E0A08000020301030200C9
:101F4300068080E0E08080000003030000030000BF
:101F5300002C3C1C068080808080800000000000F4
:101F6300000400000000000C0C00060000C0F03C60
:101F73000C0C0F030000000800F0F80868F8F000EC
:101F830000070F0B080F07000800202030F8F800A7
:101F930000000000000F0F0000080030380888F828
:101FA3007000000C0E0B0908080008003038888800
:101FB300F8700000060E08080F0700080000F8F884
:101FC30000E0E00000030302020F0F020800F8F82C
:101FD3008888880800000808080C0703000800C068
:101FE300E07858C8800000070F08080F07000800B2
:101FF300080888E878180000000E0F0100000008A8
:102003000070F8C888F8700000070F08090F070070
:102013000800F0F80808F8F0000000090D0F0301AC
:10202300000800000060600000000000000C0C00CD
:1020330000000800000060600000000000002C1C8D
:10204300000000070080C0E0F0F800000001030773
:102053000F000560606060000C0C0C0C000700F8BA
:10206300F0E0C08000000F0703010000076070105C
:1020730090F0600000001B1B0000000400382838AB
:10208300000000000800E0F01818F0E000000F0F57
:1020930001010F0F000800F8F88888F87000000F9E
:1020A3000F08080F07000800F0F808083830000090
:1020B300070F08080E06000800F8F80818F0E000FB
:1020C300000F0F080C0703000800F8F88888880839
:1020D30000000F0F08080808000800F8F88888882F
:1020E3000800000F0F00000000000800F0F80808C7
:1020F30038300000070F08090F0F000800F8F880B8
:1021030080F8F800000F0F00000F0F000800000810
:10211300F8F80800000000080F0F0800000800008E
:10212300000000F8F80000060E08080F070008007A
:10213300F8F880E0781800000F0F00030F0C000878
:1021430000F8F80000000000000F0F08080808005E
:102153000800F8F820C020F8F8000F0F0001000F66
:102163000F0800F8F860C080F8F8000F0F000001B6
:102173000F0F0800F0F80808F8F00000070F080830
:102183000F07000800F8F88888F87000000F0F00A8
:10219300000000000800F0F80808F8F00000070F3E
:1021A30008181F17000800F8F88888F87000000F57
:1021B3000F00010F0E0008003078C88818100000C7
:1021C300040C08090F060008000808F8F8080800BE
:1021D3000000000F0F0000000800F8F80000F8F8F6
:1021E3000000070F08080F07000800F8F80000F8C0
:1021F300F8000003070C0C0703000800F8F800C000
:1022030000F8F800010F0E010E0F0108001838E066
:10221300C0381800000E0F00010F0E00080078F8F8
:102223008080F878000000000F0F0000000800080D
:102233000888C8783800000E0F090808080004044D
:10224300FCFC00101F1F000638F8C000000000004F
:10225300030F0C0004FCFC04001F1F1000080C1EDD
:1022630092DE6C301800000301060F090F0604000C
:102273000000000000000004000000000000000057
:102283000800F2FA1818FAF200000F0F01010F0FFD
:10229300000800FAFA0000FAFA0000070F0C0C0F0E
:1022A30007000800F2FA0808FAF20000070F08080E
:1022B3000F07000800F0FA1A19F9F000000F0F01D8
:1022C300010F0F000800F8FA8A89890800000F0F30
:1022D30008080808000800080AFAF90908000008B5
:1022E300080F0F0808000800F0FA0A09F9F00000C7
:1022F300070F08080F07000800F8FA0201F9F800B1
:1023030000070F08080F07000800FAF9C382F9F85D
:1023130000000F0F00010F0F000800F8FA0101FA87
:10232300F80000070F0C0C0F07000800F8F9898A62
:102333008A0800000F0F080808080008000809F9B8
:10234300FA0A08000008080F0F0808000800F0F94F
:10235300898AFAF000000F0F01010F0F000800F83F
:10236300044444788000000F0002020201000800C8
:10237300C0E02020E0C00000070F08080F07000896
:1023830000E0E02020E0C000003F3F08080F070006
:102393000800C0E02020E0E00000070F08083F3FEE
:1023A300000800E0E08040606000000F0F000000C4
:1023B30000000800C0E020202020000008090909CF
:1023C3000F0600080020F8F8202020000000070F67
:1023D300080808000800E0E00000E0E00000070F44
:1023E30008080F0F000800E0E00000E0E000000331
:1023F300070C0C0703000800E0E000C000E0E00069
:10240300030F0C030C0F03080060E08080E0600002
:10241300000C0E03030E0C000800E0E00000E0E0F7
:1024230000002327341C0F03000800F9F98A8A8A65
:102433000800000F0F0808080800FF1EB3FF1EC4A2
:10244300FF1ECDFF1EDAFF1EEBFF1EFBFF1F0CFF5F
:102453001F1DFF1F22FF1F2BFF1F34FF1F43FF1FE3
:1024630050FF1F57FF1F64FF1F6DFF1F7AFF1F8B56
:10247300FF1F9CFF1FADFF1FBEFF1FCFFF1FE0FF0E
:102483001FF1FF2002FF2013FF2024FF2035FF2030
:1024930046FF2055FF2060FF206FFF207EFF20872F
:1024A300FF2098FF20A9FF20BAFF20CBFF20DCFFED
:1024B30020EDFF20FEFF210FFF2120FF2131FF210F
:1024C30042FF2153FF2164FF2175FF2186FF2197DE
:1024D300FF21A8FF21B9FF21CAFF21DBFF21ECFF68
:1024E30021FDFF220EFF221FFF2230FF2241FF2288
:1024F3004AFF2257FF2260FF2271FF227AFF2283C5
:10250300FF2294FF22A5FF22B6FF22C7FF22D8FF96
:1025130022E9FF22FAFF230BFF231CFF232DFF23B6
:102523003EFF234FFF2360FF2371FF2382FF23938B
:10253300FF23A4FF23B5FF23C6FF23D7FF23E8FF11
:1025430023F9FF240AFF241BFF242C0CF0F8FCFEC4
:10255300FE0E8EFEFEFCF8F0FFFFFFFFFFF81FFFED
:10256300FFFFFFFF0F1F3F7F7F70707F7F3F1F0FB6
:102573000C000070707078FCFCFEFEFE0000000092
:10258300000000FFFFFFFFFF000000000000007FCE
:102593007F7F7F7F000C00F0FCFCFE0E0EFEFEFC36
:1025A300F8F000000080E0F8FEFFFF3F1F03007813
:1025B3007E7F7F7F7F73707070000CF0FCFCFEFEEB
:1025C3000E0EFEFEFCFCF0C1C1C1C1DD1C3CFFFFD1
:1025D300FFF7E30F3F3F7F7F70707F7F3F3F0F0C1D
:1025E300000080F0FE3EFEFEFEFE0000E0FCFFDF8A
:1025F300C3C0FFFFFFFFC0C00707070707077F7FB1
:102603007F7F07070CFEFEFEFEFE0E8E8E8E8E0E65
:102613000E8F8F8F8F8F0303FFFFFFFFFE0F3F3F51
:102623007F7F70707F7F3F3F0F0CF0F8FCFEFE0E44
:102633000E7E7E7C7C70FFFFFFFFFF0607FFFFFF20
:10264300FEFC0F3F3F7F7F70707F7F3F3F0F0C008B
:102653001E1E1E1E1E1EFEFEFEFEFE00000000E0ED
:10266300F8FFFFFF1F07000060787F7F7F1F0700D1
:102673000000000CF0FCFCFEFE0E0EFEFEFCFCF067
:10268300E3F7FFFFFF1C1CFFFFFFF7E30F3F3F7F55
:102693007F70707F7F3F3F0F0CF0FCFCFEFE0E0E41
:1026A300FEFEFCF8F03F7FFFFFFFE060FFFFFFFF50
:1026B300FF0E3E3E7E7E70707F7F3F1F0F02707065
:1026C30000000E0E020C040CFEFEFCF8F0E0C080CD
:1026D30000000000FFFFFFFFFFFFFFFFFF7E3C182E
:1026E3007F7F3F1F0F070301000000000E040C1E35
:1026F3001E0C00000000000000000E00C0FEFEFEE5
:10270300FE1EFEFEFEFEC00000E0FFFFFFFF87800F
:1027130087FFFFFFFFE0007F7F7F7F070707070734
:102723007F7F7F7F000CFEFEFEFEFE1E1EFEFEFC74
:10273300FCF0FFFFFFFFFF1E1EFFFFFBFBF17F7F90
:102743007F7F7F78787F7F7F3F1F0D0CFEFEFEFE2D
:10275300FE1E1EFEFEFCFCF8FFFFFFFFFF0000FF56
:10276300FFFFFFFF7F7F7F7F7F78787F7F7F3F1F24
:102773000BFEFEFEFEFE1E1E1E1E1E1EFFFFFFFFA5
:10278300FF3C3C3C3C3C007F7F7F7F7F78787878C0
:1027930078780B0C0D05080DFEFEFEFEFE00C0F85A
:1027A300FEFEFE3E06FFFFFFFFFF7FFFFFFFF780FA
:1027B30000007F7F7F7F7F00030F7F7F7F7C700A16
:1027C300FEFEFEFEFE0000000000FFFFFFFFFF0015
:1027D300000000007F7F7F7F7F7878787878110C06
:1027E300FEFEFEFEF88000FEFEFEFEFEFFFFFFFF84
:1027F300FF1FF8FFFFFFFFFF7F7F7F7F7F00011F2A
:102803007F7F7F7F0CF0F8FCFEFE1E1EFEFEFCF8B1
:10281300F0FFFFFFFFFF0000FFFFFFFFFF0F1F3F62
:102823007F7F78787F7F3F1F0F0C0C0CFEFEFEFE30
:10283300FE1E1EFEFEFEFCF8FFFFFFFFFF1E1EFF37
:10284300FFFFF7E37F7F7F7F7F00007F7F7F7F7FB7
:102853000DF0FCFCFEFE1E1EFEFEFCFCF800838752
:102863008F9F9F3F7F7EFCF8F8F0C00F1F3F7F7F55
:102873007878787F7F3F3F0F0C1E1E1EFEFEFEFE04
:10288300FEFE1E1E1E000000FFFFFFFFFFFF0000F5
:10289300000000007F7F7F7F7F7F0000000C0F150B
:1028A3001EFEFEFEFEC00000FEFEFEFEFE0000C099
:1028B300FEFEFEFE1E001FFFFFFFFF00FFFFFF03E4
:1028C300FFFFFF00FFFFFFFF1F0000001F7F7F7F51
:1028D3007E7F7F0100017F7F7C7F7F7F1F00000D54
:1028E300063EFEFEF8E000C0F8FEFE3E060000C015
:1028F300FFFFFF3FFFFFFFC00000707E7F7F1F01D0
:1029030000011F7F7F7E700D0A001E1E1EDEFEFE6D
:10291300FEFE7E0080F0FEFFFFFF1F0300787F7F37
:102923007F7F7F78787878FF254EFF2573FF259882
:10293300FF25BDFF25E2FF2607FF262CFF2651FFBB
:102943002676FF269BFF26C0FF26C7FF26C8FF2645
:10295300C9FF26CAFF26EFFF26F0FF26FDFF272823
:10296300FF274DFF274EFF2773FF2795FF2796FF6E
:102973002797FF2798FF2799FF279AFF27C2FF274B
:10298300E1FF27E2FF2807FF282CFF282DFF282E31
:10299300FF2853FF287BFF28A0FF28A1FF28A2FFC1
:1029A30028E2FF290AFF290B0B013C2424242424B9
:1029B3002424243C000B013C3C3C3C3C3C3C3C3C44
:1029C3003C000A0200FE020202020202FE00007F35
:1029D3004040404040407F000A0200FEFEFEFEFEF3
:1029E300FEFEFE00007F7F7F7F7F7F7F7F001002E0
:1029F30000000000C0F0FC1E1EFCF0C00000000040
:102A0300C0F0FCFFFFFFFFC8C8FFFFFFFFFCF0C0E3
:102A13001E040000000000C0C00000181800001FC2
:102A23000204081F000018180000C0C000000000C6
:102A33008040404C8C0000000000000000000000BB
:102A430000000000000000000000CC4C40400304E4
:102A530004646300000000000000000000000000A8
:102A6300000000000000000067650505000000008D
:102A7300000006060030300000B8A8A8E8000030C7
:102A83003000000606000000000010020000008075
:102A9300E0F8FEFFFEF8E0800000000060783E3FB3
:102AA3001F1F0F0F0F1F1F3F3E7860001002030F01
:102AB3003EFEFCFCF8F8F0F0E0E0C0C08000607877
:102AC3003E3F1F1F0F0F0707030301010000100202
:102AD300030F3EFEFCFCF8F8F8FCFCFE3E0F03007F
:102AE30000000000030F3F7F3F0F030000000000C2
:102AF300100280C0C0E0E0F0F0F8F8FCFCFE3E0FEE
:102B03000300000101030307070F0F1F1F3F3E7858
:102B13006000100200008080C0C0F0FCFFFFFCF0EA
:102B230080000000030307070F0F0F1F1F1F3F3F06
:102B33007F7C70801002C0C0E0E0F0F0F0F8F8F89D
:102B4300FCFCFE3E0E010000010103030F3FFFFFEB
:102B53003F0F010000001002010E3EFEFCFCF8F8DE
:102B6300F8F0F0F0E0E0C0C0000000010F3FFFFF0D
:102B73003F0F030301010000100200000080F0FC7E
:102B8300FFFFFCF0C0C08080000000707C7F3F3FEF
:102B93001F1F1F0F0F0F0707030320040000000070
:102BA300000000000080C0E0F0F8FCFEFCF8F0E05C
:102BB300C080000000000000000000000080C0E0B2
:102BC300F0F8FC1E1FFF0FFF03132B130303030374
:102BD3000303FFFEFCF8F0E0C080000000000103E7
:102BE300070F1F3C7CF1F0F7E0E0E0E0E0E6E9E905
:102BF300E6E07F3F1F0F0703010000000000000015
:102C03000000000000000103070F1F3F1F0F070311
:102C1300010000000000000000000000200400008C
:102C23000000000000000080C0E0F0F8FCFEFCF8AB
:102C3300F0E0C08000000000000000000000008001
:102C4300C0E0F0F8FC1E1F0FFF03132B1303030355
:102C5300030303FF0F1E1CF8F0E0C0800000000018
:102C63000103070F1F3C7CF0F7E0E0E0E0E0E6E95A
:102C7300E9E6E0F7703C1C0F0703010000000000C9
:102C830000000000000000000103070F1F3F1F0F9B
:102C93000703010000000000000000000000200402
:102CA30000000000000000000000000000C0F0F879
:102CB300F8F0C00000000000000000000000000069
:102CC300000000000000000000C0F0FCFFFF030351
:102CD3000303FFFFFCF0C000000000000000000041
:102CE3000000000000C0F0FCFFFFFFFFFFFF60607B
:102CF3006060FFFFFFFFFFFFFCF0C000000000006B
:102D030000000000070F0F0F0F0F0F0F0F0F0C0C1A
:102D13000C0C0F0F0F0F0F0F0F0F0F07000000000A
:102D23001803FC02010101010181C1E1F1F9F9F18B
:102D3300E1C181010101010102FCFF000000040661
:102D4300070707FFFFFFFFFFFF0707070604000052
:102D530000FF3F40808080808080809F9F9F9F9F57
:102D63009F80808080808080403F1803FC020101A7
:102D730001E1E1E1E1E1E1E1E1E1E1612101010100
:102D8300010102FCFF00000000FFFF7F3F3F7FFFC8
:102D9300FFFFFCF8F0E0C080000000FF3F408080B0
:102DA30080818080808080808183878F8F878381EB
:102DB3008080403F1803FC02010101010181C1E150
:102DC300F1010101010101010101010102FCFF0007
:102DD30000183C7EFFFFFFFFFF7E7E7E7E7E7E7EB1
:102DE3007E7E7E0000FF3F408080808080818387DD
:102DF3008F8080808080808080808080403F180327
:102E0300FC020101010101010101010101F1E1C123
:102E130081010101010102FCFF00007E7E7E7E7EB6
:102E23007E7E7E7E7EFFFFFFFFFF7E3C180000FF5D
:102E33003F4080808080808080808080808F8783F7
:102E4300818080808080403F1803FC0201010101E2
:102E5300012161E1E1E1E1E1E1E1E1E1E10101011F
:102E630002FCFF00000080C0E0F0F8FCFFFFFF7FE2
:102E73003F3F7FFFFF00000000FF3F4080808183D2
:102E8300878F8F878381808080808080818080800E
:102E9300403F07011C22514945221C300600000017
:102EA3000000000080C0E0E0F0F8F8FC7C7E3E3ECD
:102EB3003E3E3F1F1F1F1F1E3E3E3E3E7C7CFCF8D6
:102EC300F8F0E0E0C080000000000000000000C057
:102ED300F0F8FEFF7F3F0F07030101000000000031
:102EE300000000000000000000000080C0E0F0F9D6
:102EF300FDFF7F3F3F7FFFFEF8F0C00000E0FFFFD4
:102F0300FFFF3F0100000000000000000000000080
:102F130000000080C0E0F0F8FCFE7F3F1F0F0703B6
:102F2300010000000000013FFFFFFFFFE0037FFF00
:102F3300FFFFF8800000000000000080C0E0F0F810
:102F4300FCFE7F3F1F0F070301000000000000008D
:102F530000000000000080F8FFFFFF7F0300000374
:102F63000F1F7FFFFEFCF0F8FCFEFF3F1F0F070360
:102F730001000000000000000000000000000080CD
:102F830080C0E0F0FCFEFF7F1F0F03000000000085
:102F930000000000010307070F1F1F3F3E7E7C7CDC
:102FA3007C7CFCF8F8F8F8787C7C7C7C3E3E3F1F08
:102FB3001F0F0707030100000000000000100100BD
:102FC30000007C92107C4444447C10927C000020DE
:102FD3000400000000000000000000000000FCE20C
:102FE3008202020404080810A040A010080606008C
:102FF3000000000000000000000000000000FFFFD0
:10300300FFFEFCF8F8E4C28100000001020C30C0AE
:103013000000000000000000000078FCFEFFFFFF3E
:10302300CF870707070707070707060604040403F4
:1030330000000000183C3C3C3C3C3C3C3D3F3F3FD7
:103043003F3F3F3E3C3C3C3C3C3C3C3C3C1800004E
:1030530000120110010000000883040000000101B8
:1030630002000109092100010001222E00090222A8
:1030730000010100C0FA0904000001030000000977
:103083002100010001222E000705810308006400CE
:10309300002E06A0FF09A5A10109A609A5158025F3
:1030A3007F75089540B10209A71580257F7508959E
:1030B30008810209A91580257F750895409102C0F2
:1030C300040309041A03570049004C004C00200074
:1030D300540052004E0049004300530000001803FF
:1030E300470050005300200041004C0045005200AF
:1030F300540045005200FF30C3FF30C7FF30E100EA
:1031030099A3ADB8C2CCD6E0EBF500919293949518
:1031130097999B9EDE000000000000000000000065
:1031230000000000123B751240A6F11C12588612D3
:103133004030126C5E126E50E4F522F523F521F552
:1031430024908790F0D20C90881504F0F1F70200D8
:103153002631271246BD1249A5EF640A706A124A46
:103163004FEF604824FA7060126A8CD12C90877DEF
:10317300E07002A3E07002B136900013E054FDF05A
:10318300A20DB3920D90875BE07002A3E06003127F
:10319300792190877DE07002A3E0600890876EE05C
:1031A300FF12557C2019211254DC801C900013E07F
:1031B3006402F0126E1E126DD9513190875BE0707C
:1031C30002A3E06003127921F1F7300828201A25C1
:1031D300201B22201C1F201D1C201E19201F16C36C
:1031E3009087EFE0941E9087EEE094004005124430
:1031F3004C8002C22030081F20201C201A19201BDB
:1032030016201C13201D10201E0D201F0AF11C90D8
:103213008813E0FF1259CC1241091253EF123C02FA
:1032230090841BE070022159126BDB0200333008DB
:1032330002615990875DE004F0E0D394034002E417
:10324300F0F11C7A2F7BD2752C037D047F05716A04
:103253007871766E7871E6FFD3947850127B017D96
:103263000391777871E6FF7B3F7D07F1CB80E578AB
:103273007176037871E6FDD3940650127BFF7F6E5F
:1032830091777871E6FD7BFF7F78F1CB80E59087BE
:103293005DE07027752EFF752F127530A5F1B6917D
:1032A3006F7D037F28916D7D047F41916D7D057F47
:1032B30032916D7D067F4DB11840E490875DE064E7
:1032C300017029752EFF752F127530ABF1B691621F
:1032D3007D037F48916D7D047F37916D7D057F3040
:1032E300916D7D067F3F716AB12440E290875DE076
:1032F30064027027752EFF752F127530B1F1B691E8
:103303006F7D037F37916D7D047F4C916D7D057FCC
:1033130041916D7D067F52B11840E490875DE06472
:10332300037033752EFF752F127530B7F1B69162A6
:103333007D037F2D916D7D047F4A916D7D057F43D4
:10334300916D7D067F36716A7871E6FF7BFF7D04A0
:103353009177B11A40D8227E887F2B1265277A2C69
:103363007BA1E4F52CFDFF127A5BF1D1E493787A2B
:10337300F6F1D174019308F6E47879F67979E7C325
:10338300787B9640028136E47878F67878E6FFC356
:10339300787A9640028131E52C701DE5282FFFE4F1
:1033A30033FE18E6FD2529F195F1DFC083C082F1D4
:1033B30046E493FFEC4F8032E52C640170141279DC
:1033C30012F195F1DFC083C082F146E493FFEC5F15
:1033D3008018E52C64027019127912F195F1DFC09F
:1033E30083C082F146E493FFEC6FD082D083F080F8
:1033F30038787AE6FF18E6F98FF0A4F1D1A3A32574
:1034030082F582E58335F0F58318E6FFF164E493F2
:10341300FEEFFDE5282DFDE433FCE52929F1952D8B
:10342300F582E5833CF583EEF0787806618E787952
:1034330006617FE528787A26FFE5290826FD908432
:1034430000EFF0A3EDF0EFD3947F40069084007477
:103453007FF0EDD3940740069084017407F0227A3D
:103463002F7BC0752C037D027F50716A7A2F7BC03E
:10347300752C032275F080EDF1982FF166E04BF087
:1034830022F11C787376037873E6FFC3947D50159D
:103493007B017D0191777873E6FF7BE07D06917771
:1034A30078730680E2787376027873E6FDC3940638
:1034B30050177BFFE4FFF1AD7F7FF1AD7F7EF1AD70
:1034C3007F7D917778730680E07BFF7D01E4FF9138
:1034D300777B3F7D06E4FFF1D87F0191777B607DA9
:1034E300067F01F1D87F0291777BE07D067F029111
:1034F300777BFC7D017F7FF1A67F7F91777BFE7DCC
:10350300017F7EF1A67F7E91777BFF7D017F7DF139
:10351300A67F7D8177716A7871E6FF7BFF7D0591D8
:10352300777871E6FF7BFF7D069177787106E6D3A6
:10353300947822F1E8F11C908835E07002A3E070E2
:103543000C1263F7908835EEF0A3EFF022201B45B1
:103553007A887B2B7D167FBC7E02D1156030E4D147
:103563001F602BD21B123F4F12416A715A12465AE7
:1035730090876EE0C4540F75F00AA4126F1395F090
:1035830040077F097EB012465E30B74C80FBE4D122
:103593001F70458040201C247A887B2B7D167F2C4E
:1035A3007E01D115600FE4D11F600AD21C12465A66
:1035B30012465A8023E4D11F701E8019201A197AEB
:1035C300887B2BD10F6009E4D11F6004D21A8008D5
:1035D300E4D11F7003126DD9908835E07002A3E027
:1035E30060167A887B2B127904E4D11F6007E47F8D
:1035F300FFD1207003126DD9301B10123F4F1241BF
:103603006A715A787112098B1267FD227D5A7F0FF6
:103613007E0012600378711209C474FFFFFEFDFC83
:1036230078711209A7C3020967F1E890878FE0FF59
:10363300A3E004F0C39F4002E4F0126DFAFF908709
:1036430090E0FE044F9000E0F0D2AFEE25E0247F3F
:10365300F582E43487F583E0FFA3E090878DCFF014
:10366300A3EFF0F11C126101EF4E6028D21DC21EC0
:10367300C21F7E877F657C887D371267DD12465ABD
:103683001278891267FD12410990876EE0FF126E6E
:103693006F20B7FD90877DE07002A3E06069301D65
:1036A30066201E2E7A877B657D167F2C7E01D115C1
:1036B3006019E4D11F6014D21E787112098B12674E
:1036C300FD90876EE0FF126EC48023E4D11F701E4D
:1036D3008019201F197A877B65D10F6009E4D11FF8
:1036E3006004D21F8008E4D11F7003126E1E7A8714
:1036F3007B65127904E4D11F6004D11D7003126E3F
:103703001E1278891267FD22F583E4740193FA741B
:103713000293F9120A1E120026E47876F6E478750D
:10372300F67875E6FFD3947F500D08E6F1952FF1F7
:1037330066E4F0180680EA787606E6B408DFE4FD6E
:10374300FF8141E0FC08E6FFED8FF0A4852B828525
:103753002A83A3A32582F582E58335F0F583787860
:10376300E62582F582E43583F583222582F582E41A
:103773003583F583740193FEEFFDE52C2DFDE433D2
:10378300FC908798E07A002DFDEA3CFC90879CE052
:10379300252D75F080A42400F582E5F03480F583AF
:1037A300E5822291777BFF7D062291777873E6FD90
:1037B3007BFF227531FF75321A75337BFBFD7F0169
:1037C30012417F7871766E22917778710622852B6C
:1037D30082852A832291777B017D01222FF582E561
:1037E300833EF58322E4FFFEFDFC78710209C412D7
:1037F3000026E11C300C3C908815E025E025E044D0
:1038030022F597E59730E0FB908815E0FF146008F8
:1038130004700B90880D800390880AE596F0EFC33F
:1038230094015008908815E004F08005E490881511
:10383300F0C20C22E4900005F0900003F090000722
:1038430074FFF0E4900009F09000137407F0900007
:10385300157402F090001714F09000B07438F090D3
:1038630000B47430F09000C77401F0228C6F8D7037
:10387300E4FEF9BF0104F18E8010BF0204F17E80E3
:1038830009BF0304F16E800251AB74A0F011DEEBAB
:10389300F053038011DE127A24B503047E01800500
:1038A300BC20027901EE7003EC60E9E96401702841
:1038B30011DEE05480B503027E01BF01059025555A
:1038C3008013BF0205904555800BBF0305906555D6
:1038D300800390855574F0F0AF0622857082856F62
:1038E30083228F658B688A69896ACEECCECFEDCF50
:1038F3008E6D8F6EE56C156CAE6B7002156B4E6042
:103903002E12778B7002056914F9120731FBAD6E25
:10391300AC6DAF65116F056EE56EAE6D7002056D32
:1039230014F5828E83E0FF908461E02FF080C5223E
:1039330090849EE0600221C490841CE024FD600218
:1039430021C490849DE0FE7032EFD394014072EF66
:1039530024FFFDE434FFFC908420E0FAA3E0FBC3E2
:103963009DEA9C5008CCEACCCDEBCD8004EF24FF3C
:10397300FD789EEDF6EE0408F6801BEFFDC3908400
:1039830021E09D31C55005A3E0FF8000789EEFF64E
:1039930090849DE008F690841D12772D789FE6248D
:1039A3009EF9E43484FA7B0118E6756B00F56C111B
:1039B300E5789E1277FC700990841CF0A3E0FF5118
:1039C3009022908420E09400228F6590849CE06094
:1039D30037E5656002418F90845C7405F090841C28
:1039E300E090845DF09000E0E090845EF09000E26F
:1039F300E090845FF078DF7C847D017B017A8479B9
:103A03005C7E007F4002070B90841CE024FC705E08
:103A1300E5657020C3908421E0940731C55005A368
:103A2300E0FF80027F07789EEFF6756501E49084DE
:103A3300DFF08016C3908421E0940831C55005A3BC
:103A4300E0FF80027F08789EEFF690841EE0FEA3DD
:103A5300E0FF74DF256512771D789EE6756B00F530
:103A63006C12775A1277FC702390841CF022E4784E
:103A73009FF6789FE6FFC394085011E5652F24DF76
:103A8300F582E43484F583E4F00680E622BF010482
:103A9300F18E8010BF0204F17E8009BF0304F16E32
:103AA300800251AB74F0F02290855574AAF0908A8D
:103AB300AA7455F0908555229115AB207D007C208A
:103AC3007F01710690880BE0FB7D017C207F0171F3
:103AD3000690881AE0FB7D027C207F0171069088A6
:103AE30016E0FB7D037C207F017106908813E0FBC9
:103AF3007D047C207F017106908812E0FB7D057CAC
:103B0300207F018C298D2AE4FEF9BF0104F18E8008
:103B130010BF0204F17E8009BF0304F16E800251DD
:103B2300AB74A0F0F12DEBF0530380F12D127A2446
:103B3300B503047E018005BC20027901EE7003EC1D
:103B430060E9E964017028F12DE05480B503027E39
:103B530001BF01059025558013BF0205904555808F
:103B63000BBF0305906555800390855574F0F0AF46
:103B73000622902000E0F52030003DE490880BF011
:103B830090881A7408F0908816740AF0E4908812EA
:103B9300F0908813F0908814740DF0C201C202C231
:103BA30000126B4D7D007C207F019115126B4651F5
:103BB300BB127A747102D1FF902000E0F520A3E0DC
:103BC30090880BF0902002E090881AF0902003E098
:103BD300908816F0902004E0908813F0902005E080
:103BE300908812F0902006E0908814F0783B7C8750
:103BF3007D017B017A6079007E007F0402070B3030
:103C0300090F7D007C207F0151BB127A747102C2BF
:103C130009228C298D2AE4FEFDBF0109F18EF126CC
:103C2300902AAA801FBF0209F17EF126904AAA803A
:103C330013BF0309F16EF126906AAA800751ABF115
:103C430026908AAA7455F0F12D7430F0F12D127A72
:103C53001ABB80047E018005BA20027D01EE700349
:103C6300EA60E9ED64017028AB04530380BB800272
:103C73007E01BF01059025558013BF020590455570
:103C8300800BBF0305906555800390855574F0F054
:103C9300AF0622E47872F6301102C14090841BE033
:103CA3006002C14012371C1257D875321B75336C32
:103CB3001250DF125734126DFA4401F0D2AF1237AB
:103CC300F7300119752EFF752F0F7530451279E8FE
:103CD300125E2D90873BD159125F368014752EFFEB
:103CE300752F0F7530521279E890873BD159125FC7
:103CF300981277A87B027D03E4FF12417F7872E676
:103D030064017BFF7A1B79E87028F1341279A712DA
:103D1300417F7BFF7A1B79E8127930FFC3743A9FA6
:103D2300FF752A017B3A7D03125801F1421278D7BD
:103D33008022F1341279A7F167F1451278D77BFF1E
:103D43007A1B79EC1279302443FB752A017D037FBA
:103D530043125801752EFF752F0F75305F7531FFB4
:103D630075321C75332B1277947B047D03E4FFF1CA
:103D730067F14575320F75336A7B047D58E4FFF1B3
:103D830067752F0F75306C7531FF75321C753334C1
:103D9300907FFFE493FFC4540FF534EF540FF535D0
:103DA3007B057D03E4FFF167752F0F75307975315E
:103DB300FF75321C75333D7B067D03E4FFF16775A8
:103DC3002F0F75307E9080001209977811120978B1
:103DD300EF541FFFE48F311209977816120978EF19
:103DE300540FFFE48F32120997781A120978EF54AF
:103DF3003FFFEF24D0F534E43407F5337B067D3FF2
:103E0300E4FF12417F301208E47872F6C21280098F
:103E130030130678727601C213A210E433FF78726E
:103E2300E67E00B401027E01EE5F600C126B4D1260
:103E33006B469115D1FFC210124109819A22787203
:103E4300E6FE08E690D80475F00A1209DCEE75F078
:103E53000AA42583F583E0FCA3E0FDA3E0FEA3E031
:103E6300FF22301602C1FE12371CD2169087DF12D2
:103E73004FD31278B0D1591268CE908837D1599068
:103E8300874D126B3FD1599087511209D0908837D3
:103E9300D159908743126B3FD1599087471209D06C
:103EA300127A529087DFD159908722126A79F8905B
:103EB30087DFD1591208C7908729F19E9087DFD1F8
:103EC300591208C7124FF5AF0590872AEDF19F905D
:103ED30087DFD1591208C7908728EBF09087FAE063
:103EE300908726F19F908722D1591208C7124FF568
:103EF300908727EDF0127A8C12371C22E4FBFD7CAD
:103F0300607F037106E4FB7D017C607F037106E43F
:103F1300FB7D027C607F037106E4FB7D037C607F95
:103F23000361067480F074AAF022852A82852983AE
:103F33002212000EEF75F006A4FFC3743B9FFD75BC
:103F43002EFF752F0E7530BF7531FF22752EFF754D
:103F53002F007530067531FF75321A7533EEE4FBA9
:103F63007D1E7F0112417F752EFF2290655574AA35
:103F7300F0906AAA7455F09065552290455574AA3D
:103F8300F0904AAA7455F09045552290255574AA8D
:103F9300F0902AAA7455F090255522EFF0E47B6443
:103FA300FAF9F8228C658D66E4FEFDBF0109F18EF6
:103FB300F126902AAA801FBF0209F17EF126904ABA
:103FC300AA8013BF0309F16EF126906AAA800751F4
:103FD300ABF126908AAA7455F08566828565837451
:103FE30030F0856682856583127A1ABB80047E0170
:103FF3008005BA20027D01EE7003EA60E5ED6401FD
:104003007028AB04530380BB80027E01BF0105907F
:1040130025558013BF0205904555800BBF030590BE
:104023006555800390855574F0F0AF0622C2AFD278
:10403300A8C2B8C289D2885389F0438902758CAD6E
:10404300E4F58AD2B9D28CD2A9F5C8D2BD75CD63B5
:1040530075CB6375CCC075CAC0D2ADD2CAC299C282
:104063008E43878053890F438920758DECD28E90C0
:10407300851FF0908520F0759850C299C298D2ACF4
:10408300D2BC75913075950343972075948875B1AB
:104093000875B20775B30875B40775A131D2AF437C
:1040A300A7102290881A1254D49088161270C51142
:1040B300E112718912773675E10275EA3875EA18EB
:1040C30075EC0C75EB2875E6BA75E6BE75EB2275D3
:1040D300E9BF75EE80F5E875B70143A701227F01BB
:1040E30012583C8021752F1A7530647531FF753273
:1040F3001C753351908841E0F534A3E0F5357B0519
:104103007D05E4FF317FE4FF125858E47875F678B3
:1041130075E6FFC39408504E125864E47876F67837
:1041230076E6FFC394805039EFC394405009C2C56B
:10413300D2C4EF7011800BD2C5C2C47876E6B44006
:1041430005E4FF125873D297C2C2D2C67876E6FF4F
:1041530018E61237952F123766E012585D0806806D
:10416300BE78750680A922752F007530067531FF5C
:1041730075321A7533F47B027D1E7F018F2B8D2CD4
:104183008B2DE4908797F0A3F0A3F0A3F0787576D6
:104193002908762AF540754100754231852E4385FD
:1041A3002F448530458540468541478542487B01FC
:1041B3007A8479021219DE12783DFF70026111E5EB
:1041C3002B705EEF24E0908799F0A37406F0E4A3CC
:1041D300F0F19B400241FE908798E0FDE52C2DFD18
:1041E300E433FCEE7E002DFFEE3C1279DD4002410C
:1041F300FE90879BE0F9908799E075F006A42473FD
:10420300F582E5F0341CF583E58229123766E493E1
:10421300FD75F080E52D1237981237DFEDF1AF8091
:10422300B0E52B6401704412783D24E0127A6424D3
:104233003DF582E5F034241277D9E490879BF0F1C1
:104243009B502012781F501B12785E35F0F583C007
:1042530083C08290879BE0FFD082D08312376EF1B8
:10426300A680DCF1D3640270D141FEE52B640260C9
:104273000241FE12783DFF64206049EF24D0127A98
:1042830064242AF582E5F034291277D9E490879BD8
:10429300F0F19B502012781F501B12785E35F0F519
:1042A30083C083C08290879BE0FFD082D083123784
:1042B3006EF1A680DCF1D3640370D190879AE02479
:1042C30002F0803790879A740E1277F5E490879BFB
:1042D300F0F19B5021EE252CFFE433FE908798E00C
:1042E3007C002FFFEC3E1279DD500B12378F123713
:1042F300DFE4F1AF80DBF1D3B403D190879AE0FF21
:10430300908798E02FF0908797E004F021BAE52B8F
:104313007008908798F1CC048012E52B908798B4AD
:104323000106F1CC24028004F1CC2403FD023441C4
:104333008F277A2E7B95752C037D037F6712336A53
:10434300E527C4540F30010E7E00540FFF12555F52
:104353008E318F32800312796E752EFF752F1A7589
:1043630030337B037D6FE4FF317FE527540F14B4B3
:10437300070040028141904380126EB97302439556
:104383000243AA0243C80243E6024404024422024F
:104393004431752EFF914275321A7533AAE4FB310D
:1043A3007B7A2B7B9D813E752EFF914275321A7568
:1043B30033B1123F61914275321A7533AA31797A5A
:1043C3002C7B1F8076752EFF914275321A7533C68A
:1043D300123F61914275321A7533BB31797A2C7B66
:1043E300A18058752EFF914275321A7533CE123F54
:1043F30061914275321A7533C631797A2C7BA1806B
:104403003A752EFF914275321A7533D6123F619178
:104413004275321A7533DC31797A2C7BA1801C7595
:104423002EFF914275321A75333AF1DB800D752EEA
:10443300FF914275321A753343F1DB1233652275EE
:104443002F1A7530377531FF22908843E0FF20E73C
:104453000520E602A19212371C908843E0FDC45464
:104463000F908847F0ED30E71220E40720E504546D
:104473003060089088477408F0C220908843E05465
:104483000F908845F0700204F07A2C7BA1752C0301
:10449300E4FD7F0212336AB1937532197533A3E4D5
:1044A300FB7D26123F65B1967532197533A9E4FB7E
:1044B3007D647F01317F300116752EFF752F1975CD
:1044C30030AC125F50FD12556A8E318F32800C75FD
:1044D3002EFF752F197530B3125F2B3179908847F2
:1044E300E024FB607914605414602F146002A18DE2
:1044F300B1937532197533BAF194123F67B196755A
:1045030032197533C07B047D487F02317F2020063A
:104513007F22F18D8068F1878064B19375321975BC
:1045230033C4F194123F67F1E87D6E7F02317F203F
:1045330020067F21F18D8002F1878042B19375328D
:10454300197533D0F194123F67F1E87D647F02312E
:104553007F2020067F20F18D8002F1878020B19398
:104563007532197533D7F194123F67F1E87D647F93
:1045730002317F2020067F1FF18D8002F1873109F0
:104583007FC07EC67D2D7C00E13A12371CC22022FB
:10459300752EFF752F197530A07531FF2290884154
:1045A300E0FAA3E0FBC39433EA94034002C13A90D8
:1045B3008837123E5990D800127A49F1C5F5831213
:1045C3006B3F123E5990D804127A49F1C5F5831214
:1045D30009D090883FE0C374809480500B1260F63A
:1045E300AF05ED24B4FF800890883F1260F6AF0555
:1045F300126E0C90D80875F00A1209DCECF1C5F5BF
:1046030083EFF090D809127A40F1C5F583E4F09076
:104613008842E004F07006908841E004F0126E03D3
:10462300126C9C126DAC75321A7533FD7B02123F0E
:104633006511E87F0A8012126DAC75321B75330564
:104643007B02123F6511E87F187EB0D15E7F407E0A
:104653004B7D4C7C00E13A7F1D7EB0300214D37455
:10466300189F74B09E500BEF941EEE94B050037FCE
:1046730000227876A60608A60720B7FDD2B5C2B4F5
:10468300C2B60000E47875F61267E4EE30E704D2B0
:10469300B48002C2B4C2B5EF25E07977F7EE3319DF
:1046A300F70000D2B50000787506E6B410DAC2B49C
:1046B3000000D2B630B7FD7F0122752EFF752F1390
:1046C3007530B07B017D13E4FF123F67752F1375BF
:1046D30030B97B027D117F02123F67752F1375304E
:1046E300C17531FF75321C7533027B057D133105AE
:1046F300200208F1877F0CF12E8000F1807C00F10D
:104703003A908846E0601E7F1FF17C7C00F13A7F7F
:1047130020F17C7C00F13A7F21F17C7C00F13A7F2F
:10472300227EB0D15E126B5802371C7EB0D15E7F01
:10473300C07EC67D2D7C008F2B8E2A8D298C28E48C
:104743007F207E4EFDFCAB2BAA2AA929A828C312E1
:1047530009674024E47B207A4EF9F8AF2BAE2AADEB
:1047630029AC281208C790880E1209D090880E121F
:104773003E59EC4D4E4F70F4227EB0D15E7F807E69
:10478300847D1E227F1B7EB0C15E7EB0D15ED220AF
:10479300227B04E4FD7F022290879AE0FFA3E0FEE0
:1047A300C39F222DF582E5833CF583EEF090879B32
:1047B300E004F022E6FE08E690D80875F00A120934
:1047C300DCEE75F00AA4258322E0252CFFE52D22DB
:1047D30090879CE004F0E022E4FB7D197F01317FA8
:1047E3007A2C7BA122752F197530CC908845E0F582
:1047F300317B04221257342109C0E0C0F0C083C0CA
:1048030082C0D075D000C000C001C002C003C00484
:10481300C005C006C007C2A878AA760020B20878EF
:10482300AAE6D3942340F578AAE6D3942350211122
:1048330070EF601C1170EF60171170EF6012117050
:10484300EF600D1170EF600811B39088467405F0A6
:10485300D2A8D007D006D005D004D003D002D0010F
:10486300D000D0D0D082D083D0F0D0E032E478AA88
:10487300F630B20878AAE6D3942340F578AAE6FF87
:10488300C3940E4028EFD394145022E4F620B208C8
:1048930078AAE6D3942340F578AAE6FFC3940040B0
:1048A30009EFD3940650037F01227F00227F002269
:1048B300E4FF7E01FDE478AAF630B21278AAE6FCA2
:1048C300D394235009EC942340EF7EFF80EBEF2534
:1048D300E0FF78AAE6FCC3940B400BECD394115091
:1048E300054307018013ECC39404400BECD3940AF3
:1048F30050055307FE80027EFFE478AAF620B20833
:1049030078AAE6D3942340F578AAE6D39423400209
:104913007EFF0DED6408709DEEF46010908843EF08
:10492300F0E0C4540F7002C2207F01227FFF22C037
:10493300D075D008C28C78AA06D28CD0D032C0E011
:10494300C083C082C0D075D01030981EC2989085A5
:104953001FE02401FFE433FE908520E06F7001EE39
:10496300600890851F3176E599F0D0D0D082D0834E
:10497300D0E032E0FF04F074212FF582E43485F5B2
:104983008322908520E0FF90851FE0C39F70037F03
:10499300FF22C2AF9085203176E07872F6D2AFE67F
:1049A300FF2231857871EFF6F4600FE6FF600B901C
:1049B3008621E0FE04F031DFEFF07871E6FFF4606A
:1049C30006EF6003B40ADB908621E0600C2421F536
:1049D30082E43486F583E0FF227FFF2274222EF5E2
:1049E30082E43486F58322127A8490879504F090CA
:1049F3008621E024FBFF908795E0FEC39F5015A31B
:104A0300E0FF31DFE0FEEF6E908796F0908795E050
:104A130004F080DB908796E0FF127161908621E0BD
:104A2300241FF582E43486F583E0B5071C9087964E
:104A3300E0FF127173908621E0241EF582E4348630
:104A4300F583E0B507037F01227F0022787176FFAB
:104A5300752AFF752B00752C69752D00752E067B45
:104A6300017A8679221218F5EF701A31EAEF601590
:104A73005192EF600C78717606201609123E65801C
:104A830004E47871F6E4908621F07871E6FF22E47D
:104A9300FFFEFDFC7872F1E5FC7876F1E5FC787AAF
:104AA3001209C47E867F22127946B102127946B179
:104AB300211203CB9087951209D0908795123E5906
:104AC3009087DF1209D01278F59087DF123E599054
:104AD300875E126A79F89087DF123E591208C790F1
:104AE3008763EFF0E070037418F0123FA09087DF44
:104AF300123E591208C7F1F5AF05908764ED123FD6
:104B03009F9087DF123E591208C7908762EBF078B7
:104B1300A6E6FE08E6FFB186908799B113B19B1212
:104B230055761279847800C000787212098BD00010
:104B3300F1ED787612098BE412038D127A371201A4
:104B4300691267EC12027212141E7BCE7A6379DE4D
:104B53007842120169B1AC120272B19B12016990E1
:104B6300872D1209D012793912083CC004C005C040
:104B730006C007787212098BD003D002D001D0008F
:104B8300125F811279B2C004C005C006C007B1A389
:104B9300120169D003D002D001D0001200789087AF
:104BA3009AB17590879EB113B19B12557612798491
:104BB3007800C000787212098BD000F1ED127939B8
:104BC30012083CC004C005C006C007787212098BE6
:104BD300D003D002D001D000125F811279B2C00499
:104BE300C005C006C007B1A3120169D003D002D02B
:104BF30001D00012007890879FB1759087A3B113FD
:104C03001203CBAD07AC06E41203927B187A097941
:104C1300ED1255749087A4EEF0A3EFF04E600BE015
:104C23002405F09087A4E03400F01278F5B10278FF
:104C3300A6A60608A6079087A4E07002A3E0700A60
:104C43009087F0E09087A6F0802778A4E6FE08E638
:104C5300FF78A7E624FFFD18E634FFFCB13B127989
:104C6300627C017D6812079BECC313ED139087A64A
:104C7300F078A6B1151203CB9087A71209D09087BD
:104C83009EE0B4530F90879A123E5912037C90878B
:104C93009A1209D09087A3E0B4570F90879F123ED2
:104CA3005912037C90879F1209D0C208908799E01C
:104CB3006441704878DF7C877D017B017A87799531
:104CC300FE7F1612070B9087E4123E599088371225
:104CD30009D09087E9123E5990883B1209D09087FA
:104CE300F0E090883FF0E4A3F0D2089087DFF1D39F
:104CF3001278B0123E591268CE7F01227F00220F34
:104D0300EFAC0670010E14F5828C83E0B42CF02214
:104D1300F008E6FE08E6FF78A4A60608A607B10297
:104D230078A6EEF6FC08EFF6FD78A4E6FE08E6FFAB
:104D3300ED24FFFDEC34FFFC8E278F288C298D2A70
:104D430078AB7C877D017BFF7A3179187E007F0FFA
:104D530012070BC3E52A9528FFE5299527FEAA2705
:104D6300A9287B0178AB7C871277257A8779AB02F8
:104D730019581209D078A6E6FE08E6FF78A4A6061D
:104D830008A607B10278A6A60608A60778A4E6FE39
:104D930008E6F5828E83E022E4FBFA797A784422EE
:104DA300787612098BE412038DE4FBFA7961784576
:104DB30022E47872F608F6301102E1A490841BE035
:104DC3006002E1A4127855752F0E7530EA7531FF34
:104DD30075321A7533F4E4FB7F0112417F908841E9
:104DE300E07002A3E0701B752A017B7FFDFF125068
:104DF300EE123F4275321C7533167B047D19E4FFB6
:104E0300E15C752EFF752F0E7530FA7873E6240179
:104E1300F53218E436F531E4FB7D661250E1F1A575
:104E2300123E4AF1AF120311787260025007F1A7E4
:104E3300123E4A8008F1A7123E4A12037CB1AC121B
:104E430078E6F1A5123E4AF1AF1203119087DD60B7
:104E5300025015F1B712083CE412038DC004125F2F
:104E63007AF1A5123E4A801FF1B712083CE41203FF
:104E73008DC004C005C006C007F1A5123E4A120347
:104E83007CD003D002D001D00012789DF1A5123E50
:104E93004AF1AF1203117F53600250027F4E8F31EC
:104EA300752EFF752F0F753000F1C6F5371277AAEF
:104EB3007B02F1DE123E41F1AF1203117872600200
:104EC3005005123E438006123E4312037CB1AC12DE
:104ED30078E6123E41F1AF1203119087DD60025074
:104EE30013F1B712083CE412038DC004125F7A1267
:104EF3003E41801DF1B712083CE412038DC004C08B
:104F030005C006C007123E4112037CD003D002D075
:104F130001D00012789D123E41F1AF1203117F5769
:104F2300600250027F458F31752EFF752F0F75304C
:104F330019F1C6F5371277AA7B04F1DE78721247AE
:104F4300B7F583E075F002127971752EFF752F0F97
:104F53007530327B067D077F0112417F1247F730A0
:104F63001317D37873E6940018E69400400708E615
:104F73001618700116C213A1BA201202A1BA9088A2
:104F830042E024FFFF908841E034FFFEC37873E6DC
:104F93009F18E69E50070806E618700106C212A184
:104FA300BA227872E6FE08E690D80022E4FBFAF90A
:104FB300F874F022E0FEA3E0FFE4FCFD7B107A0E20
:104FC300F9F8229087DDE0F532A3E0F5339087C24C
:104FD300E0FCA3E0FDA3E0FEA3E0227D077F010246
:104FE300417F1209C4E4FFFEFD221208C77876024E
:104FF30009C47C007D6402079BC0E0C0F0C083C08D
:1050030082C0D075D008C2CF90880CE4F0E5C0F41C
:10501300540325E025E0FFE590F454034FF0E0FF4F
:10502300908819E0FE6F6021EF600E908817E4F01E
:1050330090872004F0A374F4F0908817E0C394964B
:10504300502FEE602C42228028EE6025908720743A
:1050530001F0A374F4F0908817E0FFC39496500214
:10506300800CEFB4960BD214EE4222908817E00422
:10507300F090880CE0908819F0908720E07002A3EC
:10508300E0600E908721E024FFF0908720E034FF5A
:10509300F0908809E004F0E0C394324004E4F0D2D5
:1050A3000C90880E123E59EC4D4E4F601C90880EAA
:1050B300A3A3A3E024FFFFEE34FFFEED34FFFDECDA
:1050C30034FFFC90880E1209D0908846E0600214E9
:1050D300F0D0D0D082D083D0F0D0E032E4FB7F0197
:1050E30012417F752A017B7FE4FDFF7874A6077860
:1050F30074E6D39B503CE52A7017719E1237982FA4
:10510300123766E0440271DB123766E04440F080F8
:105113001CE52A640170167874719E1237982F1259
:105123003766E0F471DB123766E0647FF07874066B
:1051330080BD22301102413290841BE06002413273
:105143009087DCF0F1D875321B75335B11DFE4789F
:1051530072F651435040EF75F003A424C7F582E47F
:105163003487F583E0FD71CBFC513375F011A42432
:1051730044F9741012795412417F7872E6FF513466
:10518300FE9087D8E0FDEEB5050771CBFBF12AD180
:10519300CA78720680BC1247F730133B718190873F
:1051A300D8E0D39400402CE014F0E47872F6514335
:1051B300500E513371A5B50602718F78720680EED9
:1051C3007188600FE47872F651435007513314F03D
:1051D3000680F5C213803C30123971819087D8E084
:1051E300C39402502CE004F0E47872F65143500E5D
:1051F300513371A5B50602718F78720680EE7188FE
:10520300600FE47872F651435007513304F006807F
:10521300F5C21220100221361237F29087D8E075BA
:10522300F003A42489F582E4341012370B213622CB
:10523300EF75F003A424C6F582E43487F583E022F6
:105243007872E6FFC3940322301102616890841BD5
:10525300E060026168908720E07002A3E070026161
:1052630068E49087DCF0123F4275321B75331BFBF9
:10527300FD7F0112417FE47871F67871E6FFD394E4
:105283007F50097B407D011237CB80EEE47871F6C5
:1052930071795038EF71BCFDEF71ADFC716975F038
:1052A30012A424D8F9740F12795412417F7871E64D
:1052B300716A7196B50610E6FE71BCFFEE71ADFD25
:1052C300752A017B7F11EE78710680C41241093083
:1052D300133B71819087D9E0D39400402CE014F004
:1052E300E47871F67179500E71697196B5060271A1
:1052F3008F78710680EE7188600FE47871F67179AA
:105303005007716914F00680F5C213803C301239DE
:1053130071819087D9E0C39405502CE004F0E478C0
:1053230071F67179500E71697196B50602718F78B5
:10533300710680EE7188600FE47871F67179500719
:10534300716904F00680F5C212201002414B123736
:10535300F29087D9E075F003A42477F582E4341042
:1053630012370B414B22EF75F003A424CFF582E4EF
:105373003487F583E0227871E6FFC39403227F1913
:105383007EB002465E9087DCE06401229087DC7485
:1053930001F022FF9087D9E0FEEF22E6FF75F0804F
:1053A300ED22FF9087D8E0FEEF2275F003A424D10D
:1053B300F582E43487F583E02275F003A424D0F565
:1053C30082E43487F583E022EF75F003A424C8F563
:1053D30082E43487F583E022F075F080EDA4248025
:1053E300F582E5F03480F583E5822F22300814A29C
:1053F30010B014500E9087F0E0F460057181125ED6
:1054030053C210A211B01450071237F2514B800F40
:10541300A2137212500CC212C21312371C9128121B
:10542300371C020026908400E0FD91C475321A7582
:10543300336A11DFF13430100281C090841BE070B5
:105443007C908720E07002A3E06072301214908891
:105453001AE0C3940A5004E00491D112465AC212CE
:10546300801530131290881AE0D394004004E0149E
:1054730091D112465AC213752EFF752F12753048FB
:1054830090881A1270B9123F65752F1275304D123C
:1054930070D47871F67871E6FFC3940A501A908835
:1054A3001A1270AE50067A297BDB80047A297BC5F9
:1054B3001270A678710680DD1241098139221237F4
:1054C3001C752EFF752F127530457531FF22F0D2F2
:1054D30009E090310293F5A2221278C29087EEE0A0
:1054E30030010EFCA3E0FDB16AF1F9B158F1F1808E
:1054F3000A1279F2908814E01279C71267F46050A7
:105503001279BC404720184AD3ED944AEC940150D9
:105513003791C112799C123F6591C71277B1400947
:10552300125FBDD1107D5C8004D1057D607F0112C7
:10553300417F1241097F1B12472E7F1B12472E7F8B
:105543001B12472ED218800AC2188006C218800286
:10555300C2187F0122908814E0FF7E007C007D0A40
:10556300120789AC06AD07E41203927BDB7AF97963
:105573001E783F1201690203CB8F271278C29087EE
:10558300EEE0300118FCA3E0FDB16AF1F9E527C4B0
:10559300540F7E00540FFFB15FF1F1800B1279F2CB
:1055A300E527C4540F1279C71267F460501279BC0F
:1055B300404720194AD3ED942CEC9401503791C104
:1055C30012799C123F6591C71277B14009125FBDF2
:1055D300D1107D5C8004D1057D607F0112417F1273
:1055E30041097F1A12472E7F1A12472E7F1A12473C
:1055F3002ED219800AC2188006C2198002C2197FEE
:105603000122752EFF752F137530AC7871E6F531D5
:1056130008E6F5327B0322F1D875321B75333C1152
:10562300DFF134301102C1C990841BE06002C1C9AB
:10563300301212908814E0C394215005E004F0D294
:1056430009C2128013301310908814E0D3940040E1
:1056530005E014F0D209C213752EFF752F0E7530B5
:10566300CC7B03D1CA908814E06049200113752EC6
:10567300FF752F0E7530DCF17A1279781207898065
:105683000D752EFF752F0E7530E4F17AB158125F48
:1056930048752F0E7530E07B0312417B752EFF7525
:1056A3002F0E7530E87B037D0A123F65F12D7B03D6
:1056B3007D6E8008123F42127A2E7D087F011241CF
:1056C3007F124109C126227D057F0102417F90841B
:1056D30000E0123F4175321B75337D11DFF1342039
:1056E300114490841BE0703E301206F172C21280A6
:1056F30007301304F172C213752EFF752F0F753027
:105703008A7B037D05123F65752F0F7530987B05E6
:10571300D1CA200106F12A7B038004F12A7B05D13B
:10572300CA12410980B922752EFF752F0E7530C636
:1057330022E47874F67874E6FFD3947F500C7B8070
:105743007D0712347778740680EB78747601787469
:10575300E6FDD3940750177BFFE4FF123477787488
:10576300E6FD7BFF7F7F12347778740680E022A208
:1057730001B39201D209227B037D467F0102417F5F
:10578300F1D875321B7533AE11DFF134201145901A
:10579300841BE0703F301207127A7CC212800830FB
:1057A3001305127A7CC213123F4275321B7533A75D
:1057B3007B03F1EA30020B123F4275320F7533BEA1
:1057C3008009123F4275320F7533CB7B05F1EA1224
:1057D300410980B822908400E0FD752EFF752F0EDD
:1057E3007530C87531FF227D0A7F0102417F7871D0
:1057F300A60608A607227873A60608A607227873CA
:10580300A6077873E6FFD39B502EE52A701175F037
:1058130080ED1237982F123766E04402F08014E5CA
:105823002AB4010F787312539E1237982F123766DA
:10583300E0F4F078730680CA22D29700114F00EF8C
:10584300443E900005F000C29722D297C2C2C2C65E
:10585300D2C5D2C422114DEF44C0900005F0C297C7
:1058630022AE07114DEE44B8115D908401EEF02293
:10587300AE07D297C2C2C2C6EE4440115D90840007
:10588300EEF022E47871F67871E6FFC394FA500BD8
:1058930074222F1249E2E4F00680EC227A2A7B1369
:1058A300752C03E4FD7F6212336A9087F0E0F47095
:1058B3000221BAE0FF740BD39F501BE0C394215025
:1058C300157A2B7B3731BB700221BA752EFF752FEA
:1058D3001275304F21AD127A065022E0C39438502E
:1058E3001C7A2A7BAF752C037D017F6B31C270025A
:1058F30021BA752EFF752F1275305521AD1279FC23
:10590300501BE0C3944E50157A2B7B1531BB7002AC
:1059130021BA752EFF752F1275305B21ADF1F95049
:105923001DE0C3946550177A2A7BD1F11A31C270F6
:105933000221BA752EFF752F12753061806CF1EF5D
:105943005019E0C3947B50137A2B7B7B31BB606788
:10595300752EFF752F12753068804FF1E55019E0F1
:10596300C3949250137A2A7BF331BB604A752EFF9E
:10597300752F1275306E8032F1DB501BE0C394A893
:1059830050157A2B7B59F11A31C2602B752EFF7596
:105993002F1275307480137A2A7B8DF11A31C2600D
:1059A30016752EFF752F1275307A9087F012799045
:1059B3007D61E4FF12417F22752C037D017F691213
:1059C300336A908813E06402228F27119FC3908764
:1059D300EFE0944A9087EEE09401400F90872BE02C
:1059E300FFA3E09087EECFF0A3EFF0E5276402601A
:1059F3000261011254C475321A753388FBFDFF121C
:105A0300417F300118127A10F150FD12556A8E3120
:105A13008F3212784C752F127530C1800E127A10A6
:105A2300F12B12784C752F127530C5127A6D125402
:105A3300C475321B7533F0D1229087F0E0F4700205
:105A430041ECE0FF740BD39F5011E0C39421500B42
:105A5300752EFF752F127530C941F8127A06501151
:105A6300E0C39438500B752EFF752F127530D0415B
:105A7300F81279FC5011E0C3944E500B752EFF754C
:105A83002F127530D7806EF1F95011E0C394655031
:105A93000B752EFF752F127530DE8059F1EF501103
:105AA300E0C3947B500B752EFF752F127530E58084
:105AB30044F1E55011E0C39492500B752EFF752FFE
:105AC300127530EC802FF1DB5011E0C394A8500B1A
:105AD300752EFF752F127530F3801A752EFF752FF3
:105AE300127530FA9087F0800C752EFF752F1375A1
:105AF30030019087F01279907D0A7F02A1F7E527A4
:105B030064016002A1281254C475321B7533C77B2C
:105B130001FDFF12417F300115752EFF752F13759F
:105B23003008D12D908737123E59F1368011752EEA
:105B3300FF752F13753011908737123E59F198F185
:105B430022F1B41254C475321C75336D7B02E4FD2B
:105B5300FF123F67752F1375301A908726F12E7B3E
:105B6300027D1CE4FF123F67752F137530257531D5
:105B7300FF7532137533329087FAE0F534A3E0F5FD
:105B8300357B027D3AE4FF123F671254C775321B1F
:105B93007533F87B03D124300115752EFF752F1350
:105BA300753034D12D90873B123E59F136801175F3
:105BB3002EFF752F1375303D90873B123E59F19898
:105BC300F1227B037D26E4FF12417F1254C4D11CD2
:105BD300300115752EFF752F13753046F150FD12E8
:105BE300556A8E318F32800B752EFF752F137530EA
:105BF3004EF12B7B04F1AD908729F16A12787490F2
:105C03008728E0FFE4FEEB2FF15F90873F1209D076
:105C1300908763F16A127874908762E0FFE4FEEB89
:105C23002FF15F90871C1209D090873FD14790874F
:105C33001C124FD3C39BFFEE9AFEED99FDEC98FC2B
:105C43009087571209D01254C475321C7533677B81
:105C530005D124908737123E59EC4D4E4F603930B1
:105C63000115F1D11279D2D14712083C908757D14F
:105C730047D12AF1368018F1C71279D2D1471208D9
:105C83003C908757D147D12A1208C7E412038DF1FC
:105C9300227B057D2CE48010300104F1D18002F1D8
:105CA300C7E4F5317B057D2CFF12417F1254C47587
:105CB300321B7533437B06D12412797830010D12E0
:105CC3005563F148752F13753046800B120789F120
:105CD30048752F1375304E7B06F1AD1254C47532DF
:105CE3001B7533FC7B07D124908400E02405FD75EC
:105CF3002EFF752F1375306A9087F8E0F531908782
:105D0300F7E0F5327B07E4FF123F67752F13753019
:105D1300747531FF75321375337F1277947B077D6A
:105D23004BE4FFA1F71254C475321B7533C7E4FB70
:105D3300FDFF12417F300115752EFF752F1375304E
:105D430083D12D908737123E59F1368011752EFF7E
:105D5300752F1375308B908737123E59F198F122C6
:105D6300F1B41254C475321B7533437B02D12490B2
:105D73008814E0FF602630010D12555DF148752F40
:105D8300137530938010908814E012796E752EFF8E
:105D9300752F1375309A7B037D3280157BFF7A1A3A
:105DA300799D127930FFC3745A9FFD1254C4127A3D
:105DB3002EE4FF12417F1254C4D11C30011DF1BDEA
:105DC300F150FD12556A8E318F327B057D2D7F0296
:105DD300123F67752F127530C18013F1BDF12B7B14
:105DE300057D2D7F02123F67752F127530C57B0627
:105DF3007D5E7F0112417F9087FAE0FF908732E05A
:105E03006F6003127A8C127A529087EEE0FFA3E060
:105E130090872BCFF0A3EFF02275321A7533887B6E
:105E230004E4FDFF02417F1208C7E47BE87A03F92B
:105E3300F8221209DCEE75F00AA42583F583120912
:105E430097908837E0F8A3E0F9A3E0FAA3E0FB22F8
:105E5300908841E07002A3E07002E10B127A841291
:105E63006E03908795E0FCA3E0FDC39FEC9E400288
:105E7300E10B90D800127A40123E517B1C7A3479A0
:105E83004F78C0120078D14474F01203114069F1C5
:105E93001290D800123E4A7B1C7A34794F78401214
:105EA3000078D14474F01203116002504BF1129048
:105EB300D804123E4A7B927AB1798978C0F1A6D18F
:105EC3004774F01203114030F11290D804123E4A85
:105ED3007B927AB179897840F1A6D14774F01203A5
:105EE3001160025013908796E02401FF908795E09C
:105EF3003400FE126D028013908796E004F0700662
:105F0300908795E004F0C1621245A0E4FEFF229061
:105F13008795E0FEA3E022752C037D017F6A228F23
:105F2300348E338D328C31229087EEE0F531A3E04D
:105F3300F532221208C7E412038D7BDB7AF9791E4E
:105F4300783F0201698E318F32752EFF229087EEE2
:105F5300E0FCA3E02278711209A7EF2BFFEE3AFED3
:105F6300ED39FDEC38FC22E0FF7E007C0E7D101243
:105F73000789E4FCFDA804A905AA06AB0722C3EF21
:105F83009BFFEE9AFEED99FDEC98FC787A1209C41A
:105F9300787A12098BE412038DE4FBFA797A784458
:105FA30002027212007890883B227D32E4FF0241A4
:105FB3007F7B017D2CE4FF02417F752EFF752F133C
:105FC3007530A122752EFF752F1375306022752E43
:105FD300FF752F13753056229087F0E0FF7492D32C
:105FE3009F229087F0E0FF747BD39F229087F0E09D
:105FF300FF7465D39F229087F0E0FF744ED39F22F6
:106003008E27127A5BE4FFFEFDFCD1E2D1F0D1E2F0
:106013007145788EA607E6FFF4604B90883FE0FB5E
:10602300AD29116FEF603CD1B3F583F1C450081172
:10603300FAED24B4FB8008D1B311F4AF05AB0778B4
:106043008EE6FFAD29116FEF6016AE27AF28E4FC93
:10605300FD788AF17E5005788A02098B74FF8007E8
:10606300E48004E48001E4FFFEFDFC228F2CAA05FA
:10607300D1C9C364809480500811FAED24B4FF8021
:1060830006D1C911FAAF05788FA607EA252CFFE4DC
:1060930033FEC364809480500811FAED24B4FF806A
:1060A3000BE52C2AFFE433FE11FAAF057890EFF6E7
:1060B30018E6FEB507037F01227890E6FFEED39F33
:1060C300401B18E6D39B5006EBC394B44009E4D3BA
:1060D3009B5007EB9F50037F01227F0022788FE6BE
:1060E300D39B500A08E6FFEB9F50037F01227F00FA
:1060F30022F583E0FF7E007C007DB40207F0F18D82
:10610300D18B08A60608A607E4081278C5B1DD08F6
:106113001209C4B1DD7882124FE5FC78861209C4F6
:10612300B1EF787AEEF608EFF6D39414EE940050BC
:1061330004F18D8009787BE624EC7977F185D18BA6
:1061430024ECFDEE34FFFC787AE6FA08E6FBC39D07
:10615300EA9C40097878A60608A607800AEB24146F
:106163007879F6E43A18F690878DE07002A3E07030
:10617300026141EB4A700261417878EAF608EBF676
:106183007876A60208F6D37877E6940118E69400A9
:1061930040297F1C7E347DCF7CC1125E441200787F
:1061A3007876B1E41209DCEA1247C5F1B0600C401D
:1061B3000A7877E6161870011680CB7878B12090AC
:1061C300878EE09F90878DE09E40277F1C7E347DE5
:1061D300CF7C41125E441200787878B1E41209DC76
:1061E300EA1247C5F1B0500A787906E6187001063D
:1061F30080C9787AF1F660087877E6161870011688
:1062030090878DE06E7003A3E06F6008787906E6EF
:1062130018700106F1E4787AA60608A607787AB121
:1062230020787996EE18965070B1E8EF1247C1B115
:10623300CB90877BE0B4EE02F19E7E877F737C88F0
:106243007D37D1F0787E1209C47E877F73D1D5F470
:10625300603DB115603990877BF1C4500811FAEDA8
:1062630024B4FB800990877B11F6AF05AB077875E3
:10627300E6FFB11A6019D1AB1236254012D1AB1229
:1062830009C4787AE6FE08E6FF08A60608A607789A
:106293007B06E6187001068084787DE61846700256
:1062A3006141E47F207E03FDFC7882F17E40026140
:1062B30041787CE6FE08E69080081247BEB1CB9099
:1062C300877BE0B4EE02F19E7A877B737D0F7FBC00
:1062D3007E02110378861209C4B1DD788612362551
:1062E300605CE4FFFEFDFC788612362560509087E3
:1062F30090E0FFE4FCFDFE7BCC7A0CF9F812083C3D
:10630300EF787D26FFEE1836FE787AF608EFF690E2
:10631300877DE06E7003A3E06F6023787AE6FF0861
:10632300E690877DCFF0A3EFF07A8779737B0178CE
:10633300657C87B1D490877DE0FEA3E0FF22E4FE75
:10634300FF22F1A7852F82852E83125E478F828ECF
:1063530083123E59120074788FF1CE125E47F1BA60
:10636300123E5712007478931209C4789312098B62
:106373001277A8788F12098B121882F1EC12016937
:10638300127A37120272125F78E4FFFE7DE17C43DA
:106393001200741203CB7897EEF608EFF6D19450FF
:1063A3000D18D1BDED2468FFEC3401FE800B789706
:1063B300D1BDECC313FEED13FF7897A60608A6071D
:1063C300E4FFFEFDFC7893D19B700DFFFEFDFC788E
:1063D3008FD19B70037FFF22D1A3D1947D00500204
:1063E3007D01ED600811FAED24B4FF8006D1A311FD
:1063F300FAAF0522908841E07002A3E07002A10E7B
:10640300E47875F608F67875B120126E469E500250
:10641300A10E90D80075F00AEF123E4D7B1C7A3422
:1064230079CF78C1120078125E4474F012031150D0
:1064330002A1047875124FA7123E4A7B1C7A347965
:10644300CF7841120078125E4474F0120311600495
:106453004002A1047875123E437B927AB1790978A0
:10646300C2125FA6125E4774F01203115002A10418
:106473007875123E437B927AB179097842125FA60E
:10648300125E4774F0120311600250757875124F53
:10649300A71247BEAF82FE7C887D3771457877A609
:1064A30007E6FFF4605BB11560577875E6FE08E612
:1064B300FF1247BBF583E0C374809480501490D8D7
:1064C3000875F00AEF1247C111F4AF05ED24B4FBD0
:1064D300800B78751247B711F4AF05AB077877E6F1
:1064E300FFB11A601C7875124FA71247BEFAA98232
:1064F3007B01782B7C88B1D4E4908834F07876E102
:1065030095787606E6187001068109126DD9E4FEC6
:10651300FF2290883FE0FB7D16116FEF22E6FE0815
:10652300E6FFD322D1D590883FE0D39F4012EF24DA
:10653300B4FFE433FEE0FDC3EF9D7877F6EE800E03
:1065430090883FE0FF7875E6C39F7877F6E4940080
:1065530018F67876B120740B9FE49E500FC3EF9426
:1065630021EE940050067A2E7B4B80527876B12030
:1065730074219FE49E500FC3EF9438EE94005006AD
:106583007A2E7B0180387876B120747B9FE49E500D
:106593000FC3EF9492EE940050067A2D7BB7801EC2
:1065A3007876B12074929FE49E500FC3EF94A8EEC7
:1065B300940050067A2D7B6D80047A2D7B23752CF5
:1065C30003E4FD7F6702336AFAA9827BFF78737C59
:1065D300877D017E007F0A02070B74FFFFFEFDFC2F
:1065E30022E6FA08E690800875F00A22E4788AF633
:1065F30008F6D18B24FF788DF6EE34FF18F6EF4EB4
:106603007002C187788CE6FE08E6FF788AE6FC080C
:10661300E6FDD39FEC9E5068ED2FFFEC3EC313FEC7
:10662300EF13FF788EEEF608EFF608A60608F66D70
:106633007002EC6E604A788EE6FE08E6FF788D669F
:10664300700318E66E6039B1E8EF125E3574F0122C
:106653000311500B788FE624FF798DF18580A5789F
:106663008EE6FEB1E6125E3574F01203116011403E
:106673000F788FE62401798BF718E43619F78084B5
:106683007891E195E4FEFF2290878DE0FEA3E0FF81
:1066930022C3EE64809480221209A774F0020311CE
:1066A3007897E6FE08E6FF22787E12098B7882222D
:1066B300E52B2408F582E4352A22E6FE08E6FF7C72
:1066C300017D680207F0EAFFC3E52C9FFFE4940015
:1066D300FE227C887D3771457875A607E6FF227810
:1066E3008A1209C47C887D37AF2BAE2A22F1A7E436
:1066F300FFFEFDFC788F124FE5FC7893124FE5FC0B
:1067030078971209C4852F82852E83125E47852DC3
:1067130082852C83123E591200747B9A7A1979F779
:1067230078411201697893F1CE125E47F1BA123EB5
:106733005712007490872D125E47120169789712E1
:1067430009C4789712098B125F78120169C004C0DB
:1067530005C006C007789312098B125F781201698E
:10676300D003D002D001D00012007812175612794C
:1067730062788F1209C4788F02098B1209A7D3029A
:106783000967F718E634FF19F7227876760008765A
:106793000122E62401FF18E436FE2290883FE090B0
:1067A300877BF0228E2C8F2D8C2E8D2F22F583123A
:1067B30009B474F0020311E52D2404F582E4352CA9
:1067C30022E0FF7E00C374809480221209C4E52F67
:1067D3002404F582E4352EF58322D1F07871020981
:1067E300C47876E6FE08E6FF22E4FBFA79347843C0
:1067F300227871E6FE08E6FF4E22126A83752EFFA9
:10680300752F12753080125F227B057D4B7F02123C
:106813003F67752F12753085852A3485293385287E
:10682300328527317B067D767F0112417FE47F64C9
:1068330011B6500B752EFF752F12753087806B11B3
:10684300C5123FA0D31209675012E47FC811B65096
:106853000B752EFF752F1275308D804E11C5E47B9D
:10686300C8FAF9F8D31209675014E47F2C7E01119A
:10687300B7500B752EFF752F12753093802C11C5F1
:10688300E47B2C7A01F9F8D31209675014E47F9062
:106893007E0111B7500B752EFF752F12753099803D
:1068A30009752EFF752F1275309F7B05E4FD7F025E
:1068B30002417FFEFDFCAB2AAA29A928A827C3020F
:1068C3000967AF2AAE29AD28AC27225183123FA016
:1068D3001208C7EB24D0FEEA34079087F5F0A3CE65
:1068E300123F9F11C51208C7124FF59087F7EDF0BD
:1068F300517CF811C51208C79087F8EFF0517CF866
:10690300515F9087FA123F9E515F124FF59087FBBC
:10691300ED123F9F515F9087FCEBF051475403709A
:1069230018FC7D6412079BED4C70085147516AEDCA
:106933004C70069087FE741DF09087FAE0F9FF33E0
:1069430095E0FEAD2FED3395E0FCEF2DFFEE3CFE21
:10695300C3EF9418EE6480948040265150FD9087D5
:10696300F8E004F0D39D40119087F7E004F0A3E032
:10697300FD5150FCED8CF051719087FAE0252F808A
:106983002812669450299087F8E014F0940050116F
:106993009087F7E014F0A3E0FF5150FEEF8EF05123
:1069A300719087FAE0252F241875F01884800AE582
:1069B3002F2975F018849087FAE5F0F09087F5E0B9
:1069C300FAA3E0FB7C017D6DFFAE02120789AC06E2
:1069D300AD07EBAE027802CEC313CE13D8F92DFB6D
:1069E300EC3E5146124FF5C3EB9FFBEA9E514651D5
:1069F3006AEF2BFFEE3ACF2494CF34FEFE7C007D6A
:106A03000712079B9087F9EDF0787E76019087F760
:106A1300E0FF787EE6FEC39F501574FC2E5156FFAF
:106A23009087F9E02F75F00784E5F0F00680DE909B
:106A330087F9E014FF9087F8E02F75F00784A3E54A
:106A4300F0F022FA9087F5E0FEA3E0FF229087F7AB
:106A5300E024FCF582E43487F583E022AF2EAE2DEB
:106A6300AD2CAC2B0208C77C017D9002079B849060
:106A730087F8E5F0F0221209D0E47B107A27F92297
:106A83008F2A8E298D288C27221237E8200802614D
:106A93003E908837123E5990874D713F123E599070
:106AA30087511209D09087EEE07002A3E0603C7E2C
:106AB300877F4D7C877D431267DDE47FE87E03FD9E
:106AC300FC787112677E500280031237E890873B8F
:106AD300123E59125F587152908737123E59125F16
:106AE300589087371209D0D20F8034C20FA20F30CB
:106AF3000E01B3502A7146123C1590873BE0FB7D93
:106B030000123F2090873CE0FB7D01123F209087DD
:106B13003DE0FB7D02123F2090873EE0123F1D9037
:106B23008837123E59908743713F123E59908747E9
:106B33001209D0300F03D20E22C20E221209D090B6
:106B4300883B227D007C607F0322E4FFFEFDFC90F6
:106B5300873B0209D0E4F5279029AB71CF7A297BD3
:106B6300AB71BF71C740F112410971DBE4F52790A6
:106B730029B871CF7A297BB871BFE47FD07E07FD36
:106B8300FC12473A12410971C740E4752EFF752F75
:106B9300137530C87531FF75321C75330D7B057D58
:106BA3000E12410520020C7F007EB012465E30B704
:106BB3000A80FB1247807C0012473A22752C037D22
:106BC3000602336A0527E527C3940922E493FFE508
:106BD300278FF0A4240FFF22E47F107E27FDFC0201
:106BE300473A8F27E47872F6B1FA4527F0D2AF7AA5
:106BF3008079067BFFC001E52775F002A4247DF9A7
:106C0300748735F0A801FC7D01D00191579149E0CB
:106C1300FEA3E0FFF47002EEF46004EF4E700B91FC
:106C230049E4F0A3F07872F6800478727601914912
:106C3300E0FEA3E0FF90878EE02FF090878DE03E8B
:106C4300F07872E6FF22E52725E0247DF582E4341F
:106C530087F583227E007F0202070B78417C887DC3
:106C6300017B017A4079009157D1034E602AC3EF2B
:106C73009433EE940350167C007D0A120789780042
:106C83007CD87D017B017A40790202070BE490886E
:106C930041F0A3F0FFFE919C228E278F287C407D3C
:106CA300007F02123C157C407D0090884191FB7C63
:106CB300407D0190884291FBE47873F608F6AE2795
:106CC300AF287C007D0A120789C37874E69F18E613
:106CD3009E50247E40E6FA08E6FB2402FD74403A07
:106CE300FC74002BF58274D83AF58391FB78740613
:106CF300E61870010680C722E0FB7F02023B06D143
:106D03000CD39400EC94005002A191908835E0B527
:106D13000607A3E0B50702B1D1ED6F7002EC6E6018
:106D230041EF64014E603B1257F17871126520D137
:106D3300469E402E7C007D0A12078974002FF97449
:106D4300D83EFA7B01C00174F62FF974D73EA8012F
:106D5300FC7D01D0011265D6787206E61870010633
:106D630080C8908842E024FFF0908841E034FFF02F
:106D7300E0FEA3E0FF919CB1AC75321B75330B7B36
:106D830002123F651240E87F0B12464C8018B1ACEB
:106D930075321B7533157B02123F651240E87F186D
:106DA30012464C7F00227F01221234847A297BF120
:106DB300752C037D027F0A12336A908400E0240558
:106DC300FD752EFF752F1A7530617531FF22E49022
:106DD3008835F0A3F022B1D1C21BC21CC21AFFFE38
:106DE300FDFC90882BD11590882F1209D090883301
:106DF30074FFF0E4A3F022C2AF9000E0E054F82265
:106E0300908841E0FEA3E0FF22908841E0FCA3E0EC
:106E1300FD221209D0E4FFFEFDFC22E490877DF001
:106E2300A3F0C21DC21EC21FC219FFFEFDFC908744
:106E330065D1159087691209D090876D74FFF0E4CE
:106E4300A3F022908842E09F908841E022787176F7
:106E5300017871E6FFD39407501171E5EF6007786D
:106E630071E690878FF078710680E622F106940030
:106E73004043ED604014B40700503A906E84D1B99A
:106E830073026E99026E9D026EA1026EB1026EA52F
:106E9300026EA9026EAD7F0180167F0280127F040D
:106EA300800E7F03800A7F0680067F0780027F05AE
:106EB3007EB012465E2275F003A4C58325F0C58318
:106EC30022F1069400403BED14B407005034906E59
:106ED300D7D1B973026EEC026EEE026EF2026EFE51
:106EE300026EF6026EFA026EFA80007F0F800E7F4A
:106EF30010800A7F1080067F0D80027F107EB01203
:106F0300465E22EF540FFDEFC4540F75F00AA4FE42
:106F1300FFC39087EFE09F9087EEE022E47872F65C
:106F2300908813E0F630110302700B90841BE0602D
:106F33000302700B908400E0123F4175321B7533DE
:106F43002A1250DF301312908813E0D394004005C7
:106F5300E014F0D209C2138013301210908813E0AA
:106F6300C394025005E004F0D209C212752EFF1239
:106F730078CD75321B7533CF7B027D05123F6512C9
:106F830078CD75321B7533D77B047D05123F6512AF
:106F930078CD75321B7533E07B061256CA90881381
:106FA300E0700712572A7B02801A908813E0B4011D
:106FB3000712572A7B04800C908813E0B40208124E
:106FC300572A7B061256CA301038C210908813E035
:106FD3007872F612371C1234847A297BF1752C03EC
:106FE3007D027F0A12336A908400E02405123F4138
:106FF30075321C753346127A6D12410912473212EB
:10700300371C1247F7026F287872E6908813F02234
:1070130030110201A590841BE0600201A51257D82C
:1070230075321B75334A1250DF301214908816E004
:10703300C3940A5007E004F0D20911C5C21280209C
:1070430030131D908816E0D394004012E014F0D260
:1070530009E090310D93FFF5AA74FF9FF5ABC213BE
:10706300752EFF752F0F75303E90881611B9123F9C
:1070730065752F0F75304311D47872F67872E6FF79
:10708300C3940A501890881611AE50067A297BDBF8
:1070930080047A297BC511A678720680DF12410924
:1070A300011322752C037D0502336AE0FEEFC39EB4
:1070B300908400E0FF22E075F00AA4F5317B037DA4
:1070C3004B22E090310D93FFF5AAC374FF9FF5ABFC
:1070D300227B037D647F0112417F7D057F0A123489
:1070E30041E4221257D875321B7533981250DF12C0
:1070F300573420116890841BE0706230121490881A
:107103000BE0C36480948C5005E004F0D209C212F2
:10711300801530131290880BE0D36480947440057B
:10712300E014F0D209C21390880BE0FFC36480948B
:1071330080400D752EFF752F0F7530A88F31800F8E
:10714300752EFF752F0F7530B390880BE0F5317BEB
:10715300037D197F0112417F124109809522530754
:107163000FEFD39409EF50042430FF222437FF227A
:107173005307F0EFC4540FFFD39409EF50042430A6
:10718300FF222437FF22D2B5D2B6C2B4D2C32275AE
:10719300EAB022F136A3E05460701AA3E024FB6046
:1071A3000E14600D24FD600B2408700902002E806C
:1071B300DE8006615A43EA4022908821E024FE6083
:1071C3002214602D24E260561460632421707871C8
:1071D300377430F0A37454F090881CE4F0A3741255
:1071E300F0806871377430F0A37470F0903072805F
:1071F30039908820E075F003A424F9F582E5F03492
:1072030030F583E493FB740193FA740293F9908845
:1072130028EBF0A3EAF0A3E9F0120731801E7137DF
:107223007430F0A37467F0903066E493800E713786
:107233007430F0A37495F0903094E493FF90881C1D
:10724300E4F0A3EFF0800443EA4022908825E0FEB7
:10725300908824E0FDEDFF789EEEF6FE08EFF690B1
:10726300881CE0FCA3E0FDC371507F0050027F0146
:1072730090881BEFF0789E126520ED71504006A3B5
:10728300EEF0A3EFF053EA7F908828A3E0FAA3E09F
:10729300F9EA497002613190881CE0FEA3E0FF4ED9
:1072A30070067147F5EA807A78A2EEF608EFF6D316
:1072B300713F40061876000876087147FF78A3E609
:1072C3004FF5EAE478A0F608F6C379A1E778A39628
:1072D30018E66480F819E7648098501F908828E0C6
:1072E300FBA3E475F001120826A9F0FA120731F5A1
:1072F300E778A106E61870010680CE78A2E6FE08BC
:10730300E6FFC390881DE09FFD90881CE09EFCF083
:10731300A3EDF04C701590881BE06006C3EF713F3E
:107323005009908828E4F0A3F0A3F07F012275EAC6
:10733300907F002290882874FFF0A3229408EE64C3
:1073430080948022E5EA648054804430229FEE6476
:1073530080F8EC64809822908820E0D39400908891
:107363002740077404F0717480037403F075EAB066
:107373002271AE53EADF228B658A668967D3ED9467
:1073830008EC6480948040047C007D0871474DF5CF
:10739300EAED1DAE0470011C4E600FB1FB700205D7
:1073A3006614F9120731F5E780E722789E76000824
:1073B300760778A9E69087BAF0C3742496FFE41899
:1073C30096FED374079FEE6480F874809840077824
:1073D3009EEEF608EFF6789EE6FE08E6FF78A8E64E
:1073E300FC08E62422F974863CFA7B0178BB7C878F
:1073F300F1257A8779BA756A00756B087F017E007B
:10740300D104789EE6FE08E678A80826FFF618EE73
:1074130036FEF6C3EF9424EE648094804004E4F6D1
:1074230008F622C0E0C0F0C083C082C0D075D01877
:10743300E5E830E111E5EA30E609E5ED54306003B3
:1074430053EABF53E8FDE5E830E45543EA3853EA2D
:10745300DF9084DEE0FFC394405040C374409FFF3D
:10746300C39408500280027F08789BEFF69084DE75
:10747300E024DFF11DEFFD7C00717A53E8EF789B88
:10748300E6FF9084DEE02FF0C394404004F1468091
:107493000F9084DEE0FF1239CC8005B15253E8EF40
:1074A300E5E830E37AE5ED30E615B1BA789DEFF61D
:1074B30053E8F7E66069B17AEF706431968060E56E
:1074C300ED540F605490849DE0C39440504BE5ED20
:1074D300540F789BF6087600789BE6FF08E6FEC318
:1074E3009F501490849DE02E249EF582E43484F50D
:1074F30083E5EFF00680E163ED8053E8F71239335B
:10750300789BE6FF90849DE02FF0C394404010D118
:107513008F53EA9043EA20800663ED8053E8F7E552
:10752300E830E20571AE53E8FBE5E830E00353E8E9
:10753300FEE5E830E70353E87FE5E830E50653E886
:10754300DF1240B7D0D0D082D083D0F0D0E0325118
:107553008BEF702290881FE0B40515A3E0FF4480F1
:10756300F5EEEF90882760057403F080037402F052
:1075730090881F74FFF02290881EE0FEB4210DA3B3
:10758300E0B40908E490849DF07F0122EE64A170C9
:107593002390881FE0B4011C53EA7F7B017A84792E
:1075A300DF7D087C00717A9084DE7408F0FF123965
:1075B300CC7F01227F002275650175668875671E81
:1075C300E5ED540F6408600643EA407F0022E47847
:1075D3009EF608F6B1FB7002056614F9E5EF120793
:1075E30077789F06E618700106789FE664081846C8
:1075F30070E243ED807F0122AB650567E567AA660C
:10760300228E658F668B678A68896943EB28E566F6
:10761300640145657006D1834002800CE56664020F
:107623004565700AD1834006756A00756B08E47876
:10763300A0F608F6C378A1E6956BE56A6480F5F0D9
:1076430018E6648095F0501CAB670569E569AA6884
:107653007002056814F9120731F5E60806E618709A
:10766300010680D0E5EB648054804420FFE5666426
:107673000245657E0070027E40EF4E456BF5EB22BE
:10768300D3E56B9408E56A648094802290849EE03D
:107693006074B4050890849C7401F08022781C7C8B
:1076A300847D017B017A84799E7E007F4012070BE3
:1076B3007E007F407D007B017A84795C120A2490EE
:1076C300849EE024FD603224FD602514601914605B
:1076D3001B14600924087029E4F5AE801790841BFD
:1076E3007401F0E4A3F022F10AE48008F1138004AA
:1076F300F10AF11390841CF02290849FF12D123F24
:10770300A7E4FF1239CC2290849FE09000E0F0229E
:107713009084A0E09000E2F0E422F9E43484FA7B60
:1077230001227D0112070B7B0122E0FFA3E0FCA3F2
:10773300E0FD22908828E4F0A3F0A3F090881CF0E9
:10774300A3F02290849CE06002E4F090841CE0604B
:1077530005E4FF1239CC228B688A69896AE56C15C6
:107763006CAC6B7002156B4C601D0FEFCCEECC70E4
:10777300010E14F5828C83E0FDF18B700205691410
:10778300F9ED12077780D622AB68056AE56AAA6924
:107793002290880AE0FCE41203977B857AEB79C791
:1077A300783D1201698F378E368D358C34227532D0
:1077B3001A7533887B047D037F0112417F7A2E7B08
:1077C3009E752C037D017F5012336AC37872E69451
:1077D3006418E6940022F583740193FA740293AE5D
:1077E30002FF7875EEF608EFF6F5828E83E4939048
:1077F300879AF0E490879CF022E6FF7E0090841F36
:10780300E02FF090841EE03EF0C3908421E09FFFC0
:10781300908420E09EFEF0A3EFF04E22EEFDE52CD7
:107823002DFDE433FC908798E07A002DFDEA3CFCC3
:10783300D3ED947FEC6480948022908797E02402B8
:10784300F582E43484F583E0227B017D0A7F021212
:10785300417F908400E0FD752EFF2290879CE08F8E
:10786300F0A4FF7875E6FC08E68C832FF582E583A8
:1078730022A3E075F03CA4FFEB2FFBEA35F0FAED11
:1078830039F9EC38F82290876EE0FF1243337E8794
:107893007F65126527787102098B120074E4FBFA85
:1078A300797078421202729087C20209D0F52E8E47
:1078B3002D8D2C8C2B90880BE0F52F9087F122E4F3
:1078C3007871F608F608F608F622752F0E7530C2A1
:1078D3007531FF2275321B7533EC7B037D44E4FF66
:1078E30002417F1202721203CB9087DDEEF0A3EF09
:1078F300F02278A6E6FE08E6FF78A4A60608A60707
:10790300227D167F207E0312600378710209C478FA
:1079130078E62528FFE433FE08E6FD252922908733
:107923005CE024FFF090875BE034FFF02212000E4E
:10793300EF75F006A4227FA07E867D017C00787619
:107943000209A778A6EEF608EFF678A4A60608F6CD
:107953002235F0752EFFF52F8930AB047F0122E429
:10796300FBFAF9783F1200780203CB75F00AA4857D
:10797300F031F53222908814E0FF7E007C007D0A0E
:107983002278721209C47BA07A86790122E025E06D
:10799300F532E433F5317B05227532137533A57B5C
:1079A300027D032275321B7533E87B03E4FF22E477
:1079B300FBFA7970784202016908E6FC08E6FDC328
:1079C3009FEC9E2275F00AA47871A6F008F622E4D3
:1079D3007F107E0EFDFC90873722FED3EF947FEE5F
:1079E30064809480227531FF75321C75336122FEE9
:1079F300A3E07873A60608F6229087F0E0FF7438B8
:107A0300D39F229087F0E0FF7421D39F22752EFF2E
:107A1300752F127530BD22E0FCFB5420FA5303800E
:107A230022E0FD5420FCED5480FA2275321A75339E
:107A33009D7B03227BDC7A0F794978402275F00A1B
:107A4300ED1209DCEC2275F00AEB1209DCEA229054
:107A530087FAE0908732F0228F288D298A2A8B2B90
:107A630022908799F075F003A4227B027F010241E3
:107A73007F908814E0FB7D0622A202B39202D20912
:107A830022E4908795F0A3F0227F1E7EB002465E2B
:027FFE0013224C
:00000001FF
